:1080000000400020FD180100F1EA0000F1EA000044
:10801000F1EA0000F1EA0000F1EA000000000000CF
:10802000000000000000000000000000F1EA000075
:10803000F1EA000000000000F1EA0000DD85000028
:10804000F1EA0000F1EA0000F1EA0000F1EA0000C4
:10805000F1EA0000F1EA0000F1EA0000F1EA0000B4
:10806000F1EA0000F1EA0000F1EA0000F1EA0000A4
:10807000F1EA0000F1EA0000F1EA0000F1EA000094
:10808000F1EA0000F1EA0000F1EA0000F1EA000084
:10809000F1EA0000F1EA0000F1EA0000F1EA000074
:1080A000F1EA0000F1EA0000F1EA0000F1EA000064
:1080B000F1EA0000F1EA0000F1EA0000F1EA000054
:1080C000F1EA0000F1EA0000F1EA0000F1EA000044
:1080D000F1EA0000F1EA0000F1EA0000F1EA000034
:1080E000F1EA0000F1EA0000F1EA0000F1EA000024
:1080F000F1EA000001880000F1EA0000F1EA000066
:10810000F1EA0000F1EA0000F1EA0000F1EA000003
:10811000F1EA0000F1EA0000F1EA0000F1EA0000F3
:10812000F1EA0000F1EA000071E50000F1EA000068
:10813000F1EA0000F1EA0000F1EA0000F1EA0000D3
:10814000F1EA0000F1EA0000F1EA0000F1EA0000C3
:10815000F1EA0000F1EA0000F1EA0000F1EA0000B3
:10816000F1EA000059FD0000F1EA0000F1EA000028
:10817000F1EA0000F1EA0000F1EA0000F1EA000093
:10818000F1EA0000F1EA0000F1EA0000F1EA000083
:10819000F1EA0000F1EA0000F1EA000015E9000050
:1081A000F1EA0000F1EA0000F1EA0000F1EA000063
:0C81B000F1EA0000F1EA0000F1EA000032
:10840000FFFFFFFFFFFFFFFFFFFFFFFF7EF9FFFF03
:1084100010B5054C237833B9044B13B10448AFF3BE
:1084200000800123237010BD00C6FF1F0000000064
:10843000401D010008B5064B1BB106480649AFF3C5
:1084400000800648036813B1054B03B1984708BD87
:1084500000000000401D010004C6FF1F68C5FF1F8B
:108460000000000080F31188704741F238022C4B65
:10847000995841F4785199502A4A927902F00C02A5
:108480000C2A4CD041F244022749995003F5583345
:108490009A78120703D59A7842F008029A70204B16
:1084A000224941F24402995041F204015A5842F4DF
:1084B000803242F0C0025A501A6842F440221A60D8
:1084C00003F5E83324225A70194A80211170A22240
:1084D0001A70DA7802F01F02DA7007221A710C2281
:1084E0005A719A799007FCD59A79D106FCD40D4B34
:1084F0009A7902F00C02082AF9D14C225A719A7921
:1085000002F00C02082AFAD1064B9A795206FBD5E2
:1085100022221A709A7902F00C020C2AFAD17047C2
:1085200000700440004006400000330100001301C9
:1085300000500640264B5A7902F0E0025A711A792F
:1085400002F0F8021A71A3F500531A7802F08C02B7
:1085500042F050021A705A7802F09C0242F0400237
:108560005A709A7802F0E6029A701A4A0023137041
:1085700083F31188184B012283F8182383F81923F9
:10858000022283F8582383F8592383F81D2383F8A4
:108590002E2383F82F2383F8302383F831230322FB
:1085A00083F82D2383F82F2383F8312383F8332393
:1085B00083F83523042283F83923052283F83A23EC
:1085C000062283F85723072283F84923704700BF08
:1085D00000F0074000E0074000E100E0364B68464D
:1085E0001A6820F0070101328D46F1B51A60334B4D
:1085F0001A6801321A60324B1A683AB11A68013AA5
:108600001A601B6813B92F4B01221A702E4B1A687F
:1086100012B11A68013A1A602C4B2D485B682D493B
:108620009BB2036002680B689A4202680B6817DD10
:10863000D31A294C294DB3F5004FD4E9002306DAAB
:10864000D0F800C00F682E68C7EB0C0527E0D1F802
:1086500000C007682E68C7EB0C0505F5803511E0F2
:108660009A4222DA0A6803681B4C1C4DD31AB3F5F0
:10867000004FD4E900230ADAD1F800C007682E6859
:10868000C7EB0C057543521B63EBE5730BE0D0F8A9
:1086900000C00F682E68C7EB0C0505F580357543E3
:1086A000521943EBE573C4E9002303680B60BDE88E
:1086B000F1408546704700BF1CC6FF1F04D0FF1F56
:1086C00014CDFF1F10CDFF1F18CDFF1F00900340DA
:1086D00034CDFF1F28CEFF1F70CDFF1F6CCDFF1FB5
:1086E000064A41F23C03D15841F00071D150044B8D
:1086F000044A5A6007221A60704700BF00700440A5
:1087000010E000E040190100014B1868704700BFFD
:108710001CC6FF1F072888BF0020134B134A53F8BD
:10872000203010B5124CB4FBF3F441F234032D2089
:10873000D15841F48061D1500E4B4FF400725A6011
:108740009A6006F0EDF90C4B0022DA709A709A717B
:10875000DA725A71C4F30422E4B21A705C70DA78E7
:1087600042F02C02DA7010BD701B01000070044052
:1087700020AA44000090044000A00640094B1A685B
:1087800059680132202A08BF00228A4208D019689D
:10879000194408721A60044BDA7842F08002DA70E9
:1087A000704700BF20C6FF1F00A006400A4B996A11
:1087B000DA6A91420CD09A6A511C1A44996292F872
:1087C000302002709A6A202A04D100229A6201E0C5
:1087D000002070470120704720C6FF1F044B1A7805
:1087E00002F0FF0012B100221A700120704700BF92
:1087F00010CDFF1F014B1865704700BF20C6FF1F3B
:10880000684620F007018D4631B527480179C9B285
:108810008C0615D5254BDA6A9C6A0132202A08BFDE
:108820000022A24206D0DD6AC4795819E4B280F869
:108830003040DA621E4A052010601A6D1D4B1A6026
:108840004A0609D51C4B4FF400329A60A3F5152354
:10885000DA7802F0BF02DA700B0621D5154B1968E1
:10886000F1B9124B18685A68904214D0124A4FF46A
:10887000003050605A68501C1A445860107A0A4AF6
:10888000C0B2D0715868202808BF5960D37843F02F
:108890004003D37004E0044BDA7802F07F02DA7010
:1088A000BDE831408546704700A0064020C6FF1F46
:1088B00014CDFF1F18CDFF1F00F00F4062B67047A8
:1088C00072B6704762B6704772B670474FF0E023D9
:1088D00008B1034A00E0034AC3F80C2D704700BFFB
:1088E0000400FA050100FA0510B9C90801F0E6BC58
:1088F000704773B5434A444944484FF48073136149
:1089000053619363D3631364536448618860A1F532
:1089100035214FF440300B604B608B60CB608B6235
:10892000CB620B644B6401F53521403148614860EE
:10893000374938480B6040F607044B608B60CB62C8
:10894000446144603448036043608360C3600361F2
:1089500000F53320C0301424446104244460102402
:1089600084602E4C636104F5322404F58074202564
:10897000656141F204042A4D2E5926F0E0062E517D
:108980002E5946F0C0062E514FF4A064CC601360FF
:10899000D36000230A211A461B4C08256560002578
:1089A0000195019DB5F57A7F02D2019D0135F7E76A
:1089B0002469E507144C4FF00805A56048BF013253
:1089C00000250195019DB5F57A7F02D2019D013503
:1089D000F7E72469E40758BF01330139DCD10A2ADB
:1089E000104A03D10A2B01D1012300E000231370A8
:1089F000044B4FF4E0621A60DA601023436002B067
:108A000070BD00BF0090044000F00F4028800300BC
:108A100000B0044080F00F4000C0044000D004408B
:108A20000070044068CDFF1F0F4B1B7882B0CBB1A4
:108A30000E490F4B20224A609A6000220192019851
:108A40000C4A904202D8019A0132F7E720228A604C
:108A50005A6000230193019A064B9A42E8D8019B81
:108A60000133F7E702B0704768CDFF1F00F00F40F9
:108A700000F10F401FA1070007281BD8DFE800F016
:108A800004070B0D0F1214164FF4004201E04FF4CF
:108A90008032094B0DE002220AE0082208E04FF480
:108AA000006205E0012203E0042201E04FF480624D
:108AB000024B5A60704700BF00F00F4040F00F407B
:108AC00007281BD8DFE800F004070B0D0F1214165F
:108AD0004FF4004201E04FF48032094B0DE00222D6
:108AE0000AE0082208E04FF4006205E0012203E0FA
:108AF000042201E04FF48062024B9A60704700BF8D
:108B000000F00F4040F00F4038B50546002445FA0C
:108B100004F3DB07E0B202D5FFF7AEFF01E0FFF799
:108B2000CFFF0134082CF2D138BD08B506282CD867
:108B3000DFE800F0040D12171C212600002005F0CC
:108B400063FDB0F5806F34BF0020012008BD104BDD
:108B5000186900F0010008BD0D4B1869C0F38000D2
:108B600008BD0B4B1869C0F3802008BD084B18697D
:108B7000C0F3400008BD064B1869C0F3C00008BD33
:108B8000034B1869C0F3C02008BD002008BD00BF1A
:108B900040F00F4007282DD8DFE800F004090E133D
:108BA000181D2227144B1868C0F3C0307047124BB1
:108BB0001868C0F300407047104B1868C0F34000BD
:108BC00070470E4B1868C0F3C00070470B4B186815
:108BD000C0F3C0207047094B186800F001007047CF
:108BE000064B1868C0F380007047044B1868C0F348
:108BF000802070470020704700F00F4040F00F4089
:108C000038B500242546E0B2FFF78FFF18B10123E5
:108C1000A3401D43EDB20134082CF4D1284638BDE1
:108C200010F0010F314B07D05A6942F002025A612D
:108C30004FF400329A6006E04FF400325A605A69ED
:108C400022F002025A6110F0020F294A06D0596937
:108C500041F0080159610221916005E00221516053
:108C6000596921F008015961410707D5596941F453
:108C7000006159614FF40061916006E04FF40061BA
:108C80005160596921F400615961010707D559699B
:108C900041F0010159614FF48031996006E04FF4D1
:108CA00080315960596921F001015961C10606D529
:108CB000596941F0040159610121916005E00121E8
:108CC0005160596921F004015961810606D559693D
:108CD00041F480615961042393607047042151601D
:108CE0005A6922F480625A61704700BF40F00F4019
:108CF00080F00F401B4B5A6810F0010F14BF42F078
:108D0000030222F002025A60DA6881074CBF42F087
:108D1000030222F00202DA60124BDA6A10F0040F4A
:108D200014BF42F0030222F00202DA621A6801075D
:108D30004CBF42F0030222F002021A60094B9A680B
:108D400010F0100F14BF42F0030222F002029A60EA
:108D50009A6A81064CBF42F0030222F002029A6234
:108D6000704700BF00A0044020B9034B1869C0F34E
:108D7000403070470020704700F00F4008B50820D1
:108D800005F042FC5E2804D90F4B1A784AB901223B
:108D900006E0082005F038FC542802D80A4B0022CF
:108DA0001A70082005F030FC632803D9074B042211
:108DB0009A6008BD082005F027FC542802D8034B10
:108DC00004225A6008BD00BF74C6FF1FC0F00F40E8
:108DD000034B1878013801288CBF00200120704710
:108DE00074C6FF1F034B1878012806BF02221A70B1
:108DF0000020704774C6FF1FC0B201F073BBC0B241
:108E000001F064BB08B507F0ABFD06F073F806F09F
:108E100023F8BDE8084007F025BE38B5054605F043
:108E200071FF08280AD900242819013405F0EAFF47
:108E3000092CF9D106F01AF8012038BD002038BD00
:108E4000092105F07FBF002006F008BA214A41F24F
:108E50003C030120D15841F44051D1501E4B1F49D1
:108E600018601A680A431A601D4ADA601A61DA6AE1
:108E700042F08052DA621A6822F001021A601A681F
:108E800022F000621A6003F5F8334FF400721A61A1
:108E90005A619A61DA61A3F5F033186018680143EA
:108EA00019601049D96001F520011961D96A41F0B2
:108EB0008051D962196821F001011960196821F007
:108EC0000061196003F500331A605A609A60DA6035
:108ED0001A6170470070044000C00240000C1F80FF
:108EE0000300013E0400513EFF281CD800F03F0063
:108EF000214B72B141F0006141EA004058631E4BC2
:108F0000DA6A002A1946FADACA6A1B4BD000FBD586
:108F100028E041F0004141EA00405863164BDA6A0C
:108F2000002AFBDA1EE0B0F5007F22D200F03F00FD
:108F3000124B72B141F0006141EA004058630F4B9F
:108F4000DA6A002A1946FADACA6A0C4BD200FBD553
:108F500008E041F0004141EA00405863074BDA6AFB
:108F6000002AFBDA986BDA6A42F01042C0B2DA6289
:108F700070470020704700BF00C0024000D0024090
:108F8000C0EBC00038B500220C4600F50065032197
:108F90000120FFF7A9FFC5F3072100220120FFF7F9
:108FA000A3FFE9B200220120FFF79EFF00210A463D
:108FB0000120FFF799FF00210A4620700120FFF7EA
:108FC00093FF00210A4660700120FFF78DFF00210A
:108FD0000A46A0700120FFF787FF00210A46E070D3
:108FE0000120FFF781FF00210A4620710120FFF7D1
:108FF0007BFF6071012000210246FFF775FFA07121
:1090000038BD38B54FF40064012006210246FFF751
:109010006BFF052100220120FFF766FF01200021E0
:109020000246FFF761FF8307F3D5022100220120EA
:10903000FFF75AFFC4F3072100220120FFF754FF76
:109040000120E1B20022FFF74FFF0025B5F13F0EEE
:10905000DEF1000252EB0E02012000210135FFF784
:1090600043FF402DF2D1052100220120FFF73CFFF4
:10907000012000210246FFF737FFC307F3D4403435
:10908000B4F5804FC0D138BDF7B5C0EBC00000F5D6
:1090900000650C46002203210120FFF725FFC5F3E0
:1090A000072100220120FFF71FFFE9B20022012063
:1090B000FFF71AFF00210A460120FFF715FF0021E4
:1090C0000A4607460120FFF70FFF00210A46064621
:1090D0000120FFF709FF00210A4605460120FFF79E
:1090E00003FF00210A468DF803000120FFF7FCFE74
:1090F00000210A468DF804000120FFF7F5FE8DF8E7
:109100000500012000210246FFF7EEFE23788DF8CE
:109110000600BB420DD16378B3420AD1A378AB42BB
:1091200007D1DDF80300D4F80330C31A5842584180
:1091300000E0002003B0F0BD38B5044601200D4624
:1091400002460621FFF7D0FE052100220120FFF78D
:10915000CBFE012002460021FFF7C6FE8207F3D5B1
:10916000022100220120FFF7BFFEC4F307210022E5
:109170000120FFF7B9FEE1B200220120FFF7B4FEA3
:10918000012029460246FFF7AFFE052100220120FB
:10919000FFF7AAFE012000210246FFF7A5FEC30744
:1091A000F3D438BD38B50C46C0EBC00505F50060FA
:1091B0000978FFF7C1FF05F601006178FFF7BCFFF2
:1091C00005F60200A178FFF7B7FF05F60300E17886
:1091D000FFF7B2FF05F604002179FFF7ADFF05F6B2
:1091E00005006179FFF7A8FF05F60600A179BDE843
:1091F0003840FFF7A1BF2DE9F041044601200F469A
:10920000164606210246FFF76FFE052100220120C7
:10921000FFF76AFE012000210246FFF765FE850781
:10922000F3D5022100220120FFF75EFEC4F30721DF
:1092300000220120FFF758FE0120E1B20022FFF7D3
:1092400053FE0025B54242D0013414F03F08795D49
:1092500004D0721EA81A4242424100E001220120BD
:10926000FFF742FEB8F1000F2FD1731E9D422CD2A2
:10927000052100220120FFF737FE012000210246D0
:10928000FFF732FEC107F3D4012006210246FFF7A3
:109290002BFE052100220120FFF726FE01200246B9
:1092A0000021FFF721FE8207F3D5022100220120D1
:1092B000FFF71AFEC4F3072100220120FFF714FE76
:1092C0000120E1B20022FFF70FFE0135BAE70521C8
:1092D00000220120FFF708FE012000210246FFF7CF
:1092E00003FEC307F3D4BDE8F08110B503210446A3
:1092F00000220120FFF7F8FDC4F30721002201201E
:10930000FFF7F2FDE1B200220120FFF7EDFD0120A1
:1093100000210246BDE81040FFF7E6BD70B50446E7
:109320000E461546032100220120FFF7DDFDC4F3A0
:10933000072100220120FFF7D7FDE1B20120002222
:10934000FFF7D2FD0024AC420CD06A1EA31A5A4289
:109350004FF001004FF000015A41FFF7C5FD3055B5
:109360000134F0E770BD37B5052100220120FFF779
:10937000BBFD012000210246FFF7B6FD10F071048D
:10938000F2D1FFF7C1F90546FFF7BEF9401B0028EF
:10939000B8BF4042B0F5FA6F09DA4CB940F2FF703D
:1093A000FFF7A3FFB0F1AA035C425C41ECE71CB1FC
:1093B0002B4B1B78002B3CD040F2FF700021FFF7B5
:1093C000BBFEFFF71EFE002026494022FFF713FFD9
:1093D0000024B42202FB04F000F580702249FFF75C
:1093E0000AFFA01C4001214920220134FFF703FF9E
:1093F000032CEED1002301934FF4C364204601A94E
:1094000004220434FFF7F7FEB4F5FF6FF6D1002312
:1094100001934FF4A764204601A904220434FFF706
:10942000EAFEB4F5C36FF6D140F2FF70AA21FFF750
:1094300083FE00200B494022FFF770FF40200C49BB
:109440002022FFF76BFF60200A492022FFF766FF0A
:10945000802009492022FFF761FF03B030BD00BF23
:1094600068CDFF1F0CC0FF1FC01B0100A01B010027
:10947000C8CDFF1FE8CDFF1F08CEFF1F0000000072
:109480002DE9F8431378C3F3411507460E461446F9
:109490002DBB3E4A02EB451208321179F9B9D907C2
:1094A0001DD45F2B1BD83A49495DC1B913F0970908
:1094B00015D1DFF8E48018F805302BB14846517813
:1094C000FFF712FA08F80590DFF8D08018F8053099
:1094D0002BB1002001F006F8002308F805302178B0
:1094E000002240F20110FFF7FFFC3070617800228B
:1094F00040F20110FFF7F8FC7070A178002240F2F2
:109500000110FFF7F1FCB070E17840F20110012288
:10951000FFF7EAFCF0702378D80735D45F2B33D8F7
:1095200003F01E03082B11D0142B24D0062B2BD1B3
:1095300024235F430C2303FB0575164FA278E378C1
:109540003D4443EA02236B60BDE8F883A278E378E8
:1095500024214F430C2143EA022301FB05750D4AE8
:109560005351A17809070FD56FEA03536FEA1353DC
:109570005351BDE8F883242257430C2202FB0575A2
:10958000044FE3783D442B72BDE8F883C8CDFF1F3C
:1095900084CEFF1F78CDFF1F81CEFF1F87CEFF1F18
:1095A00007B513788DF8013053788DF800108DF8D9
:1095B000023001A993788DF803306A46FFF760FF07
:1095C00003B05DF804FB07B58DF800108DF801209D
:1095D0008DF8023001A99DF810308DF803306A46ED
:1095E000FFF74EFF03B05DF804FB07B500238DF8CD
:1095F00000108DF801308DF80320131201A96A467E
:109600008DF80230FFF73CFF03B05DF804FB5F29E3
:109610002DE9F34106460D46144658D811F01E07B1
:10962000C1F3411202D0022F1DD050E0032313FBDF
:1096300000223049120188188C504368C3EB040E95
:10964000BEF1000FB8BFCEF1000EBEF5000F08DB73
:109650009C42CCBF284C294C0A441C440123137360
:1096600035E0077333E00327224B17FB00273F0148
:10967000D91924F07F4EC1F808E04C6001F10800D0
:10968000D959C4EB010EBEF1000FB8BFCEF1000EE8
:10969000BEF5000F984618DBA142CCBF164B174B06
:1096A000520123448DF800201A148DF801201A125B
:1096B0008DF80220304601A96A4647448DF80330F0
:1096C000FFF7DEFE01233B7301E000230371231447
:1096D0008DF801303046231201A96A468DF80050FA
:1096E0008DF802308DF80340FFF7CAFE02B0BDE8E6
:1096F000F08100BFBCCEFF1FFFFF7F00010080FF95
:1097000007B511F01C0202D1FFF781FF0CE0002326
:109710008DF800106A4601A98DF801308DF80230ED
:109720008DF80330FFF7ACFE03B05DF804FB0121B8
:1097300040F201100A46FFF7D7BB13B541F0010113
:1097400014468DF8041001AA6946FFF799FE9DF8AA
:10975000013023709DF8023063709DF800009DF881
:109760000330A37002B010BD07B541F001018DF8C0
:10977000041001AA6946FFF783FE9DF803309DF8A7
:10978000020043EA0020030544BF6FEA00506FEA7D
:10979000105003B05DF804FB73B54901CCB244F03E
:1097A0001503164601A96A4605468DF80030FFF7F5
:1097B00067FE9DF805308DF8013044F014049DF8E3
:1097C00006308DF80040284601A96A468DF802301F
:1097D0008DF80360FFF754FE02B070BD73B5490108
:1097E000CCB244F01503164601A96A4605468DF829
:1097F0000030FFF745FE9DF805308DF8013044F04C
:1098000014049DF807308DF80040284601A96A46E7
:109810008DF802608DF80330FFF732FE02B070BDA4
:1098200037B57F236A460D4601A904468DF80030FE
:10983000FFF726FE7E238DF800309DF805308DF869
:10984000013005F00F059DF807308DF802502046D5
:1098500001A96A468DF80330FFF712FE03B030BD50
:109860002DE9F3474001C7B2C1F30A06002047F0D3
:10987000180101AAFFF761FF9DF805804FEA18194A
:1098800008F00F08C84530460FDB07F043FAC9EB74
:1098900008080446012000FA08F00D4607F04AFACD
:1098A0000022354B07F0ACFA10E007F033FAC8EBB2
:1098B00009080446012000FA08F00D4607F03AFABC
:1098C00002460B4600202C4907F0C4FB02460B461B
:1098D0002046294607F0BEFB07F0CCFC07F03CFA17
:1098E00023A3D3E9002307F08BFA07F0C3FC07F0AA
:1098F00033FA0022214B07F083FA4FF0FF39044678
:109900000D46CA464FF00008012000FA08F007F0A3
:1099100011FA02460B462046294607F071FA07F075
:1099200081FCA0F18002802A38BFC14608F10108FD
:1099300028BF5046B8F10E0F01D08246E4E700245C
:109940008DF8050047F01201204601AA8DF8044069
:109950008DF80690FFF724FE204647F00C013246B2
:10996000FFF743FE204602B0BDE8F087AFF300806A
:1099700004560E2DB29DEF3F0000604000002040D5
:1099800073B54A084FF48073032414FB0234B423E4
:1099900013FB0044054620460E46FFF7A6FC8DF853
:1099A0000400601CFFF7A1FC8DF80500A01CFFF768
:1099B0009CFC46EA45118DF80600C9B2002001AAB8
:1099C000FFF7EEFD02B070BD37B50C4641EA40111D
:1099D000054601AAC9B20020FFF7AFFE64080322C2
:1099E0004FF4807312FB0434B42313FB0544204668
:1099F0009DF80410FFF7A0FB601C9DF80510FFF711
:109A00009BFBA01C9DF80610FFF796FB03B030BD32
:109A100010B5C4B221466401E4B200200222FFF76F
:109A2000BBFE44F008010020FFF76AFE44F00A0183
:109A30000020BDE81040FFF763BE37B5400140F09D
:109A40001604E4B20D4601AA21460020FFF775FE78
:109A50009DF8053015F0010F14BF43F0400323F0CB
:109A600040038DF805309DF8053015F0020F14BF46
:109A700043F0100323F010030020214601AA8DF8C3
:109A800005308DF80600FFF78BFD03B030BD37B50C
:109A9000400140F01604E4B20D4601AA2146002020
:109AA000FFF74BFE9DF8053015F0010F14BF63F072
:109AB0007F0303F07F038DF805309DF8053015F026
:109AC000020F14BF43F0200323F02003002021469F
:109AD00001AA8DF805308DF80600FFF761FD03B08F
:109AE00030BD07B5400140F0160101F0F60101AAB2
:109AF0000020FFF722FE9DF80530C3F38010DB063F
:109B000048BF40F0020003B05DF804FB07B5400118
:109B100040F0160101F0F60101AA0020FFF70DFE4A
:109B20009DF80530D8099B0648BF40F0020003B0FD
:109B30005DF804FB70B50F4C000123189A68914240
:109B400009DD8A1AC2F18075AA425E6801DC3244DE
:109B500009E0751B0AE00ADA521AC2F18075AA42BE
:109B60005E6802DCB21A5A6001E035445D60204450
:109B7000816070BDBCCEFF1F73B541F001030C4680
:109B800001AA69468DF804300546FFF779FC9DF877
:109B900002309DF801201B0243EA02439DF8032096
:109BA00043EA02010B0248BF41F07F415F2C1CD801
:109BB000C4F3411614F01E0411D0022C15D105EB8C
:109BC0004500304421F07F41C0B2FFF7B3FF0323CB
:109BD00013FB0565064B03EB0515696805E00323D8
:109BE00013FB05652D01024B5959084602B070BDA3
:109BF000BCCEFF1F38B50C4668210546FFF7BCFFF9
:109C000014B140F0010201E020F001022846682171
:109C1000BDE83840FFF7FBBC73B51C4B587E10F015
:109C2000010004D00020682140F2231202E06821E4
:109C30004FF49172FFF7EBFC0020022300937E218A
:109C400002460346FFF7BFFC00240025E6B2E9B256
:109C500030460135FFF794FE1D2DF7D17501EDB2A9
:109C600045F00C010020FFF787FF01463046FFF763
:109C7000F7FD0134002045F0160143F2FF12FFF713
:109C8000B4FC032CE1D102B070BD00BF0CC0FF1FBB
:109C9000F0B5450185B0044645F0030303AA002052
:109CA00002A98DF80C30FFF7EBFB9DF80A109DF828
:109CB0000930090241EA03419DF80B30204619435F
:109CC000FFF738FF15482301C21802F108010E7989
:109CD0000EB3134E0C2707FB0464247ADCB9C65874
:109CE0005268B71A002FB8BF7F42B7F5000F05DBE7
:109CF0009642CCBF0B4B0C4B134401E0C3580C7184
:109D0000DAB200920020C3F3074205F0E001C3F38A
:109D10000723FFF758FC05B0F0BD00BFBCCEFF1F06
:109D200078CDFF1FFFFF7F00010080FFAFF30080B1
:109D300070B50546C5F3074100224FF48170FFF767
:109D4000D3F80B4C0602C5F3072100224FF48170B3
:109D50002660FFF7C9F830430602E9B24FF481707C
:109D600001222660FFF7C0F830430609266070BD67
:109D700078C6FF1F10B5264CC00023181A79032A95
:109D800084BF03221A7123189A79032A84BF0322FD
:109D90009A7123181A7A0F2A84BF0F221A72231875
:109DA0005A7A072A84BF07225A7223189A7A0F2AEE
:109DB00084BF0F229A72221813795279DB0343F47D
:109DC0000021E1601AB1124A43F40423D36022183F
:109DD0000F4BD2791AB1DA6842F40052DA602044AB
:109DE000037A8279DB0143EAC223E2681A43437AA9
:109DF00042EA0313C27AE3601AB9827A1343044A2F
:109E0000D360E068FFF794FFE368236110BD00BFF3
:109E100078C6FF1F10B5114C0023C000E360231863
:109E20005B7E13B14FF40073E36022180B4B927EFC
:109E30001AB1DA6842F48072DA6023182044DA7EBC
:109E40000F2A84BF0F22DA76C07EE3681843E060F1
:109E5000FFF76EFFE368E36110BD00BF78C6FF1F28
:109E600070B5C3001F4C1D1A254495F8221095F8B3
:109E7000202095F8216001294FEA8232C0EB0301CE
:109E8000214442EA063242F46022E26091F8235013
:109E900008BF42F4806201F1200108BFE260E2687D
:109EA000097942EA05220129E26003D10D4942F015
:109EB0008002CA60191A21440A4A91F82510012922
:109EC00003D1D16841F04001D1601B1A234493F8BB
:109ED0002600E36843EA0010E060FFF729FFE3682B
:109EE000A36270BD78C6FF1F10B543001C4C1A1842
:109EF00022442C3292F901103F29C4BF3F215170F6
:109F00001A1822442C3292F901103F31BCBFC121F2
:109F100051701A1822442C3291781F2984BF1F21B6
:109F200091704FF44022E2601A18224492F82C20DB
:109F3000012A03D10A4A4FF45021D160034423443B
:109F4000E26893F82E00024393F82D0000F07F00A2
:109F500042EA0020E060FFF7EBFEE368236310BDF8
:109F600078C6FF1F10B58300224C1A18224492F8BD
:109F70003410012984BF012182F834101A182244B8
:109F800034325178032984BF032151701A182244B6
:109F9000343291780F2984BF0F2191701A1822440E
:109FA0003432D178032984BF0321D1701A18224496
:109FB0003432117903440F29234484BF0F211171D6
:109FC00093F8380003F1340293F8343040F4202041
:109FD00040EAC330537840EA4330937840EA0320A4
:109FE000D37840EA4310E060FFF7A2FEE368E36342
:109FF00010BD00BF78C6FF1F214B012010B5032103
:10A000000024052283F82C0083F8250002205972D1
:10A0100083F8201083F8211018729A72DC7283F88A
:10A020002D2083F82E2083F8224083F8234083F8E4
:10A03000244083F8260083F8344083F8354083F8C1
:10A04000364083F8374083F838405C769C76DC767F
:10A0500018715C71DC719C710A4B04229A60204675
:10A06000FFF780FF2046FFF73FFF2046FFF7F8FE8F
:10A070002046FFF7CFFE2046BDE81040FFF77ABE2E
:10A0800078C6FF1FC0F00F40054B042903EBC00347
:10A0900018BF0022D97618BF5A76FFF7BBBE00BFA3
:10A0A00078C6FF1F044B03EBC003597609B10422A5
:10A0B000DA76FFF7AFBE00BF78C6FF1F024B03EB97
:10A0C000C0039976FFF7A6BE78C6FF1F024B03EBCD
:10A0D000C000C07E704700BF78C6FF1F024B03EB75
:10A0E000C000407E704700BF78C6FF1F024B03EBE5
:10A0F000C000807E704700BF78C6FF1F024B03EB95
:10A10000C0031971FFF736BE78C6FF1F024B03EB81
:10A11000C0035971FFF72EBE78C6FF1F024B03EB39
:10A12000C003D971FFF726BE78C6FF1F024B03EBB1
:10A13000C0039971FFF71EBE78C6FF1F024B03EBE9
:10A14000C0031972FFF716BE78C6FF1F024B03EB60
:10A15000C0035972FFF70EBE78C6FF1F024B03EB18
:10A16000C0039972FFF706BE78C6FF1F024B03EBD0
:10A17000C0000079704700BF78C6FF1F024B03EB99
:10A18000C0004079704700BF78C6FF1F024B03EB49
:10A19000C000C079704700BF78C6FF1F024B03EBB9
:10A1A000C0008079704700BF78C6FF1F024B03EBE9
:10A1B000C000007A704700BF78C6FF1F024B03EB58
:10A1C000C000407A704700BF78C6FF1F024B03EB08
:10A1D000C000807A704700BF78C6FF1F034A00EBBB
:10A1E0008003134483F83410FFF7BCBE78C6FF1F0A
:10A1F000034B00EB800213445970FFF7B3BE00BF5E
:10A20000ACC6FF1F034B00EB800213449970FFF7AD
:10A21000A9BE00BFACC6FF1F034B00EB8002134476
:10A22000D970FFF79FBE00BFACC6FF1F034B00EB0A
:10A23000800213441971FFF795BE00BFACC6FF1F23
:10A24000034B00EB8000184490F83400704700BFC7
:10A2500078C6FF1F024B00EB80001844407870471F
:10A26000ACC6FF1F024B00EB80001844807870479B
:10A27000ACC6FF1F024B00EB80001844C07870474B
:10A28000ACC6FF1F024B00EB8000184400797047FA
:10A29000ACC6FF1F034A00EB4003134483F82C10A5
:10A2A000FFF722BE78C6FF1F034B00EB40021344AA
:10A2B0005970FFF719BE00BFA4C6FF1F034B00EB88
:10A2C000400213449970FFF70FBE00BFA4C6FF1FE2
:10A2D000034B00EB4000184490F82C00704700BF7F
:10A2E00078C6FF1F034B00EB4000184490F90100B3
:10A2F000704700BFA4C6FF1F024B00EB400018448C
:10A3000080787047A4C6FF1F034AC0EBC003134404
:10A3100083F82010FFF7A4BD78C6FF1F034BC0EBE6
:10A32000C00213445970FFF79BBD00BF98C6FF1FC2
:10A33000034BC0EBC00213449970FFF791BD00BFFF
:10A3400098C6FF1F034BC0EBC0021344D970FFF740
:10A3500087BD00BF98C6FF1F034BC0EBC00213446C
:10A360001971FFF77DBD00BF98C6FF1F034BC0EBFF
:10A37000C00213445971FFF773BD00BF98C6FF1F99
:10A38000034BC0EBC00213449971FFF769BD00BFD6
:10A3900098C6FF1F034BC0EBC000184490F8200084
:10A3A000704700BF78C6FF1F024BC0EBC0001844C7
:10A3B0004078704798C6FF1F024BC0EBC00018449E
:10A3C0008078704798C6FF1F024BC0EBC00018444E
:10A3D000C078704798C6FF1F024BC0EBC0001844FE
:10A3E0000079704798C6FF1F024BC0EBC0001844AD
:10A3F0004079704798C6FF1F024BC0EBC00018445D
:10A400008079704798C6FF1F2DE9F0472E4DDDF883
:10A410002080099F1E462B18044693F840308A4638
:10A420009146042B1AD8DFE803F003080D12170039
:10A43000FFF7A0FC2B19012212E0FFF711FD2B19E9
:10A4400002220DE0FFF78EFD2B19032208E0FFF733
:10A450004BFD2B19042203E0FFF7DCFC2B19002233
:10A46000C4EBC4042C4483F8402094F82620164BF7
:10A47000012A12D002D3022A14D020E0BAF1000F30
:10A4800003D01B689B0C8AF80030B9F1000F16D07E
:10A490002B689B0A89F8003011E086B11B689B0A83
:10A4A00033600CE01EB11B68DB0B5B013360B8F15D
:10A4B000000F04D02B68C3F3842388F800300FB159
:10A4C0002B683B70BDE8F08778C6FF1F30B9044B9E
:10A4D000DA7A1AB90122DA72FFF74CBC704700BF72
:10A4E00078C6FF1F28B9034BD97A11B1D872FFF78C
:10A4F00041BC704778C6FF1F06281AD8DFE800F075
:10A5000004070A0D101316000A4B1B6810E0094BD4
:10A51000DB690DE0074B1B690AE0064BDB6B07E0CC
:10A52000044B1B6B04E0034B9B6A01E0014BDB7A9D
:10A530000B60704778C6FF1F13B5C84C63789A1F2D
:10A54000012A0FD98C2B0DD0C02B0BD0C72B09D0D3
:10A5500003F16002D2B2182A04D903F13402D2B254
:10A56000322A03D8A27822B10422DBE2A278022A9E
:10A57000FAD8A42B00F0658273D8842B00F01181E7
:10A5800026D8062B00F0508110D8022B00F009814C
:10A5900006D8002B00F0F380012B00F0F680C0E21B
:10A5A000042B00F0228140F2188133E1802B00F06F
:10A5B000E68007D80C2B00F03E810D2B00F05D816A
:10A5C000072BB4E0822B00F06F8140F2DE800CE1BB
:10A5D000942B00F030812AD88A2B00F071810FD89B
:10A5E000862B00F01781C0F0F880872B40F099820D
:10A5F000A178490141F00E01002001F0EE015AE17D
:10A600008D2B00F07581932B00F037818C2B40F05F
:10A610008882E178A078C1F10801C9B2FFF734FD62
:10A62000A2788F4B03EB4213E278DA727CE2A02B24
:10A6300000F0F28109D8992B00F077819A2B00F075
:10A640008781952B40F06D825AE1A22B00F0EB81BF
:10A6500000F2F081D4F80310A078C9B2FFF72EFD04
:10A6600062E2B32B00F03A8243D8AB2B00F00C82AD
:10A670001CD8A72B00F0F3810CD8A52B00F0E881A3
:10A68000A62B40F04E82D4F80310A078C9B2FFF791
:10A690005DFD49E2A92B00F0E98100F2EE81D4F8DA
:10A6A0000310A078C9B2FFF799FD3DE2AF2B00F08F
:10A6B000008212D8AD2B00F0EE8100F2F381D4F8C5
:10A6C0000310A078C9B2FFF7B1FDA278654B03EB88
:10A6D000C203D4F803205A7126E2B12B00F0F081B6
:10A6E00000F2F581D4F80310A078C9B2FFF716FE86
:10A6F0001AE2C32B00F0558122D8B82B00F00A8251
:10A700000FD8B62B00F0F18100F2FC81B52B40F0A0
:10A710000882A278524B03EB4213D4F803209A61CB
:10A7200002E2C12B00F02F8100F23481C02B40F0F7
:10A73000F881A2784A4B03EB4213E2789A72F3E174
:10A74000D22B00F0448109D8CC2B00F03281D12BE0
:10A7500000F03781C72B40F0E48165E0D62B00F094
:10A760004981FE2B00F04E81D42B40F0DA81A27893
:10A770003B4B03EB4213D4F803205A61D4E1A17898
:10A780004901002001F0E00106E0A178490141F013
:10A790000201002001F0E201D4F80320FEF737FFA8
:10A7A000C2E1A178D4F80320490141F0080100205A
:10A7B00001F0E801FEF719FFA178D4F80320490160
:10A7C00041F0060101F0E6010020002AB8BF524224
:10A7D000FEF70BFFA378012119E0A178490141F0B0
:10A7E0000A01002001F0EA0165E0A178D4F8032015
:10A7F000490141F0060101F0E6010020FEF7F5FEF7
:10A80000A378D4F80310184A42F823100021174AFD
:10A81000D15489E1D4F80310A078FFF721F8A37888
:10A82000D4F80310124AEFE7A2780D4B03EB421362
:10A83000E2785A7278E1A178490141F0140101AA45
:10A84000002001F0F401FEF778FFD4F803209DF812
:10A8500005307AB143F0020323E000BFECCEFF1FC6
:10A86000C8CDFF1F3CCDFF1F20D4FF1FBCC6FF1F5C
:10A8700014D0FF1F23F0020313E0A178490141F037
:10A88000140101AA002001F0F401FEF756FFD4F8EC
:10A8900003209DF8053012B143F0010301E023F0DD
:10A8A00001038DF8053018E0A178490141F0040159
:10A8B000002001F0E401D4F80320FEF796FE33E116
:10A8C000A178490141F01401002001F0F40101AA2E
:10A8D000FEF733FFE3788DF80630A178490141F0A7
:10A8E0001401002001F0F40101AAFEF759FE1BE15A
:10A8F000A178490141F01A01002001F0FA01DAE7DC
:10A90000A178490141F0140101AA002001F0F401ED
:10A91000FEF713FFD4F803209DF8053012B143F081
:10A920000403BEE723F00403BBE7A178490141F02B
:10A93000180101AA002001F0F801FEF7FEFEE278FE
:10A940009DF8053002F00F0223F00F03134310E0CF
:10A95000A178490141F0180101AA002001F0F80195
:10A96000FEF7EBFE9DF80530E27803F00F0343EAB3
:10A970000213A1788DF80530490141F0180100203B
:10A9800001F0F801B0E7A278684B03EB4213E278DC
:10A990001A72C9E0A378654AD4F803105B01D1505C
:10A9A000C2E0A278614B03EB4213D4F803205A6053
:10A9B000BAE0A2785D4B03EB4213D4F80320DA81AE
:10A9C000B2E0A078D4F8031004F008F8ACE0A07866
:10A9D000564BE178D4F8032003EB401301F01F013C
:10A9E0001A6103F0CDFFD4F80310A078491103F0E9
:10A9F000BFFF99E0A2784D4B03EB4213D4F803203C
:10AA00009A8391E0494AA178D4F8033002EB4112CD
:10AA100003B10123137387E0D4F80310A078C9B2FF
:10AA2000FFF740FB80E0D4F80310A078C9B2FFF72D
:10AA300065FB79E0D4F80310A078C9B2FFF766FB94
:10AA400072E0D4F80310A078C9B2FFF76FFB6BE097
:10AA5000D4F80310A078C9B2FFF770FB64E0D4F813
:10AA60000310A078C9B2FFF779FB5DE0D4F80310BA
:10AA7000A078C9B2FFF7BCFB56E0D4F80310A07869
:10AA8000C9B2FFF7BFFB4FE0D4F80310A078C9B2FA
:10AA9000FFF7C2FB48E0D4F80310A078C9B2FFF773
:10AAA000F9FB41E0D4F80310A07849B2FFF7FCFBB2
:10AAB0003AE0D4F80310A078C9B2FFF725FC33E0E0
:10AAC000D4F80310A078C9B2FFF732FC2CE0D4F818
:10AAD0000310A078C9B2FFF735FC25E0D4F80310C5
:10AAE000A078C9B2FFF742FC1EE0A078D4F803308A
:10AAF0000F4A42F83030BBB902EBC0025179FFF780
:10AB000095FB11E0A2780A4B03EBC203D4F80320B3
:10AB10001A7109E0D4F80310A078C9B2FFF7FEFA61
:10AB200002E00322034B1A7002B010BDC8CDFF1F14
:10AB30003CCDFF1F08D0FF1F37B5C74DC74C6B7802
:10AB40009A1F012A0FD98C2B0DD0C02B0BD0C72BED
:10AB500009D003F16002D2B2182A04D903F13402F9
:10AB6000D2B2322A04D8AA782AB1042323709BE2F5
:10AB7000AA78022AF9D8A32B00F0358200F2AA8025
:10AB8000832B00F05C813DD8082B00F07B8115D829
:10AB9000032B00F04A8105D8012B00F0348140F2EC
:10ABA0002C813AE1052B00F04D81C0F04881062B45
:10ABB00000F04B81072B00F05F8163E20C2B00F06B
:10ABC0006A810BD80A2B00F0868100F27381002085
:10ABD000FDF7ABFF003018BF012051E2802B00F0E1
:10ABE0000C8101D80D2B33E0812B00F00C81822BDE
:10ABF00040F04882A978490141F00401002001F0A9
:10AC0000E40119E1942B00F0468130D8872B00F045
:10AC1000708105D8852B00F0088140F2FE8011E19B
:10AC20008C2B00F06E810FD88A2B40F02B82A978F4
:10AC3000490141F01401002001F0F40101AAFEF7DE
:10AC40007CFD9DF806307CE18D2B00F06481932B18
:10AC500040F01882A978490141F01401002001F068
:10AC6000F40101AAFEF769FD9DF805303EE19C2B39
:10AC700000F031811CD8992B00F0558111D8952B0B
:10AC800040F00082A978490141F01401002001F050
:10AC9000F40101AAFEF751FD9DF80530C3F38003CE
:10ACA0004FE19A2B00F04F819B2B00F00381E9E1EB
:10ACB000A02B00F0908103D89D2B00F0E380E1E110
:10ACC000A12B00F08C81A22B40F0DC81A878FFF74B
:10ACD0004DFAD5E1B52B00F0C2813AD8AC2B00F08B
:10ACE0009E811BD8A72B00F08A8108D8A52B00F0E5
:10ACF0007E8100F28081A878FFF750FAC0E1A92B8D
:10AD000000F08581C0F07F81AA2B00F08481AB2BFD
:10AD100040F0B881A878FFF7ADFAB1E1B02B00F0B0
:10AD20008C8108D8AE2B00F0808100F28281A87857
:10AD3000FFF7CEFAA4E1B22B00F08781C0F0818149
:10AD4000B32B00F08681B42B40F09C81AB78444A51
:10AD500083E1C72B79D01DD8C02B00F08D800BD894
:10AD6000B72B00F08781C0F08081B82B40F08A813A
:10AD7000A878FFF70BFA83E1C22B00F0F880C0F04F
:10AD8000F080C32B00F0F880C42B40F07B81AA78C0
:10AD9000344BF9E0D12B00F00E8115D8CE2B00F00A
:10ADA000F18008D8CC2B40F06D81AA782E4B03EBB4
:10ADB0004213DB89C5E0CF2B00F0E980D02B40F0B7
:10ADC0006181AB78294A48E1D42B00F0F88008D89B
:10ADD000D22B40F05781AA78234B03EB42131B6917
:10ADE000AFE0D62B00F0F180FE2B40F04B81AA782B
:10ADF0001D4B03EB42131B7BA3E0A9784901002004
:10AE000001F0E00106E0A978490141F002010020CB
:10AE100001F0E201FEF7B0FE32E1A978490141F00C
:10AE20000801002001F0E80106E0A978490141F09D
:10AE30000A01002001F0EA01FEF796FC20E1AA7861
:10AE40000B4BA1E0AA780B4B9EE0AA78064B03EBD4
:10AE500042135B7A75E000BFECCEFF1F08D0FF1FE6
:10AE600038CDFF1F24CDFF1FC8CDFF1FC3CDFF1F4F
:10AE700020D4FF1F14D0FF1FAA788C4B03EB421382
:10AE80009B7A5EE00020FEF752FCAB785B00184135
:10AE900000F0010355E0A978490141F014010020B8
:10AEA00001F0F40101AAFEF748FC9DF80530C3F358
:10AEB000400346E001AA00207C21FEF73EFCAA7870
:10AEC0000223520003FA02F29DF806301A420CBF28
:10AED0000023012335E001AA00207C21FEF72DFC90
:10AEE000AB789DF806205B0042FA03F303F0010300
:10AEF00027E0A978490141F00E01002001F0EE01A0
:10AF00009AE7AB782BB90020FFF7E0F8C0F1080012
:10AF1000B6E00423B7E0A978490141F01A01002006
:10AF200001F0FA0188E7A978490141F018010020F1
:10AF300001F0F80101AAFEF700FC9DF8053003F0CE
:10AF40000F036360A0E0A978490141F018010020D7
:10AF500001F0F80101AAFEF7F0FB9DF805301B098E
:10AF6000EFE7AA78514B03EB42131B7AE9E7AB7882
:10AF70004E4A5B01D358E4E7AA784C4B03EB4213EB
:10AF80005B68DEE7AA784A4B53F82230D9E7AB7802
:10AF9000484AD05C0021616010B1474801254560F6
:10AFA000D154464AD15C19B1616841F00201616037
:10AFB0000021D15468E0A87803F004FD60E0AA788D
:10AFC0003A4B03EB42135B69BBE7AA78374B03EBC1
:10AFD00042139B8BB5E7A878FFF780F850E0A8787C
:10AFE000FFF784F84CE0A878FFF7C8F848E0A878A5
:10AFF000FFF7DCF844E0A878FFF7E0F840E0A87835
:10B00000FFF7E4F83CE0A878FFF71AF938E0A878F1
:10B01000FFF720F934E0A878FFF724F930E0AA78A8
:10B02000274B03EBC2035B798BE7A878FFF75AF94C
:10B0300026E0A878FFF7AEF922E0A878FFF7B4F988
:10B040001EE0A878FFF7B8F91AE0A878FFF7BCF976
:10B0500016E0A878FFF7C8F912E0D35C71E7AA7888
:10B06000124B03EB42139B696BE7AA78144B53F81E
:10B07000323066E7AA78124B03EBC2031B7960E714
:10B08000606001E0032323700E4B1B7863B10E4B0D
:10B0900062681A600D4B1AB91A6842F0080202E0A1
:10B0A0001A6822F008021A6003B030BDC8CDFF1F35
:10B0B0005CCDFF1FC0CDFF1F08D0FF1F57CDFF1F66
:10B0C0003CCDFF1F03D0FF1FF4CFFF1FF4CEFF1FA7
:10B0D00038B5984A9378022B144600F02381032B4D
:10B0E00000F03681002B40F0BB8153784E2B00F0EE
:10B0F000A5802BD8462B72D016D8422B60D009D809
:10B10000402B59D0412B40F0A9818B4BD17819703D
:10B11000002059E0442B5BD0452B40F09F81864BAB
:10B12000D178597105204FE04B2B77D004D8472BAD
:10B1300060D0492B66D091E14C2B7AD04D2B40F05A
:10B140008D817D4BD178597515203DE0542B00F051
:10B15000B2801BD8512B00F08E8009D84F2B77D0AE
:10B16000502B40F07B81744BD178997516202BE0E1
:10B17000522B00F08F80532B40F070816E4DD2F82F
:10B1800003302946102041F8103F8AE0832B00F05D
:10B19000BA8006D8552B00F09980562B00F0A3807A
:10B1A0005CE1852B00F0B980C0F0B280FF2B40F04D
:10B1B0005581D278614B55E140F2FF70D17803E0C0
:10B1C0005D4BD17859700120BDE83840FDF7B4BF20
:10B1D0005949D2F8033041F81C3F1C2005E056497C
:10B1E000D2F8033041F80C3F0C200422BDE838406F
:10B1F000FEF701B8504DD2F803302946082041F837
:10B20000083F4EE0D2784C4B0AB9DA7503E04C495E
:10B210000122DA754A601720D97DD5E7464CD178EE
:10B22000E1700320FDF788FFE078BDE83840FDF7C6
:10B23000E1BA414BD17899700220C5E73E4CD2F873
:10B240000300E084FDF7ECFC262021180222CDE764
:10B25000D2F80310384CC9B219206176FDF76CFFA3
:10B26000607E10F001001ABF002001210146BDE8F8
:10B270003840FEF7BFBC304B1A7D12F0010F1D465F
:10B2800004D0E378DB0701D4FDF7BBFEE178297534
:10B29000142099E72849D2F8033041F8203F2020B4
:10B2A000A3E70422FDF7A7FF687929892A8ABDE868
:10B2B000384003F0DBB9D2F80330012B00F2D08024
:10B2C0001D49D37801F81A3F1A200AE0D2F803305A
:10B2D000012B00F2C580174B1749DB7801F81B3FA3
:10B2E0001B20012282E7D2F80330124D0F2B00F20F
:10B2F000B7800020E978FEF793FA0F49EB7801F860
:10B30000243F2420EDE70F4BD2F803205A6038BDCC
:10B310000D4BD2F803201A6038BD0A4BD2F8032037
:10B320009A6038BD5178094BD2F8032043F82120A8
:10B3300038BD00BFECCEFF1F0CC0FF1F02D0FF1FA7
:10B3400008D0FF1FBCC6FF1F04D0FF1F20D0FF1F67
:10B3500053782E2B00F28280DFE803F018212A8038
:10B36000808080808033383D8080808080808080B5
:10B37000808080808080804244464D4F5180808014
:10B38000808080585D62676C71767B00364BD4F8A4
:10B3900003201A60FDF7B8F9344BD86038BD324B42
:10B3A000D4F803205A60FDF7AFF9304B186138BD6F
:10B3B0002D4BD4F803209A60FDF7A6F92B4B58616A
:10B3C00038BD294BD4F80320DA6038BD264BD4F8B9
:10B3D00003201A6138BD244BD4F803205A6138BDCC
:10B3E000002002E000200BE00120D4F80310BDE8AB
:10B3F0003840FEF722BB012002E00220F5E70220E0
:10B40000D4F80310BDE83840FEF741BB164BD4F822
:10B4100003209A6138BD144BD4F80320DA6138BD9B
:10B42000114BD4F803201A6238BD0F4BD4F8032017
:10B430005A6238BD0C4BD4F803209A6238BD0A4BCF
:10B44000D4F80320DA6238BD074BD4F803201A631E
:10B4500038BD054BD4F803205A6338BD032200E001
:10B460000422034B1A7038BD38CEFF1FBCC6FF1F25
:10B4700008D0FF1F2DE9F843044615460E46002963
:10B480004AD0002848D0814246D04FEA42185FFA9D
:10B4900088F848F0060739460020FEF76DFB48F0B3
:10B4A0000C0181460020FEF767FB8046204605F030
:10B4B000E7FF0446304605F0E3FF0146204606F06C
:10B4C000EBF80646484605F0DBFF314606F0E4F8A7
:10B4D00006F0F4F90446404605F0D2FF314606F086
:10B4E000DBF806F0EBF9002C08BF01240B4900281B
:10B4F00014BF80464FF00108304606F0B7F918B186
:10B5000028464146FEF7ACF9224600203946FEF7B0
:10B510007EF8034B01225A55BDE8F8830000A04194
:10B52000BCC6FF1F70B50C4D2B5C04469BB1C6B268
:10B530000A4B710141F0060153F82420002001F06C
:10B54000E601FEF752F8064B304653F82410FEF79A
:10B5500087F900232B5570BDBCC6FF1F20D4FF1FE9
:10B5600014D0FF1F2DE9FF41BE4FDFF814833B7855
:10B57000D7F8036088F801306422212B88F8002076
:10B58000C8F804603C46454601F09D825AD80E2B0F
:10B5900000F005872AD8072B00F0D78211D8032B9B
:10B5A00000F01C8107D8012B00F0BD80022B00F0B9
:10B5B000EC8001F065BD052B00F0BF8240F2DA801F
:10B5C000BFE20A2B00F05D8509D8082B00F0F1835B
:10B5D000092B41F05585FFF77BFD01F053BD0C2B86
:10B5E00000F0998640F2798600F0AABE182B01F08F
:10B5F000328012D8142B00F0778707D80F2B00F079
:10B60000F586132B00F0298701F03ABD162B01F0C7
:10B61000108040F28B8701F010B81C2B01F047819D
:10B6200006D81A2B01F0358041F2228001F042B891
:10B630001F2B01F08A8101F2E3811E2B00F05F864F
:10B6400001F01EBD802B01F0188338D8402B01F08B
:10B6500002831BD8242B01F091820DD8222B01F0FC
:10B660008682232B41F00C857F4B1B68C7F8033083
:10B67000FFF72EFD01F006BD262B01F0B582C1F0CB
:10B68000AA82272B01F0D58201F0FABC442B01F0ED
:10B69000EB8208D8422B01F0E18201F2E28202F053
:10B6A0009EF901F0EFBC462B01F0E482C1F0DF828D
:10B6B000472B41F0E58402F098F901F0E3BC872BB9
:10B6C00001F0AA8316D8832B01F001830AD8812BBD
:10B6D00001F0E882822B41F0D384644B02221A7677
:10B6E00001F0D0BC852B01F02283614B41F20E8327
:10B6F00001F021BB8C2B01F0E48309D8892B01F0E8
:10B70000B283C1F054838A2B01F0C48301F0B8BC2A
:10B71000F22B01F06784FF2B01F0A9848D2B41F0FF
:10B72000AF8401F0F5BBB97802292AD84F4B01222A
:10B730005A54504B00255D544F4B284602225D540D
:10B74000FEF72AF8B978490141F00601284601F0D0
:10B75000E60140F2FF72FDF748FFB978D7F8032001
:10B76000490141F00801284601F0E801FDF73DFFDD
:10B7700001F088BCB87802284CD93A4B5B78022B90
:10B7800048D004232B7001F07DBCB978354E0229D6
:10B79000F7D8364B01225A54364B00245C54364BB2
:10B7A000204602225C54FDF7F7FFB178490141F0D1
:10B7B0000601204601F0E60140F2FF72FDF715FF99
:10B7C000B178D6F80320490141F00801204601F084
:10B7D000E8015242FDF709FF01F054BCB878022895
:10B7E000CFD802F0B7FE02220020B978FDF7D4FFCF
:10B7F000B978490141F0080101F0E8010020FDF7A6
:10B800007FFFBB78194A0121D1541B4A0021D15432
:10B8100001F038BC6378032B00F28B81DFE813F072
:10B82000040032005C005301FFF77CFEA178124B4C
:10B8300000255D540F4B5D54104B012218788A404F
:10B8400020EA020249011A702846D4F8032001F0C8
:10B85000E001FDF7DCFE2846A1782A46FDF79CFFB3
:10B8600001F010BCECCEFF1FF4CFFF1FBCC6FF1FC2
:10B870000CC0FF1FC0CDFF1F57CDFF1F31CDFF1FD5
:10B8800008D0FF1FFFF74EFEA378B94A0026D65412
:10B89000B84AD6545B0143F0020101F0E2013046A0
:10B8A000FEF76AF9B44BD4F80370A178074401227B
:10B8B00018788A4020EA020249011A70304601F0E5
:10B8C000E0013A46FDF7A3FE3046A1783246FDF787
:10B8D00063FF6F6001F0D6BB142E3FF752AF10F03C
:10B8E000C00724D102283FF64CAF06EB46060644BB
:10B8F000A24B53F82650FFF715FEA1789C4B5F54DE
:10B900009C4B5F549C4B012218788A4020EA02022B
:10B9100049011A7038462A4601F0E001FDF777FE2A
:10B920003846A1783A46FDF737FF01F0ABBB402F10
:10B9300040F0978000250195029503952B4640FA2B
:10B9400003F2D20706D504AA2A440135032D02F8D2
:10B95000103C02D00133032BF1D10027AF421DDA96
:10B960001DF807804046FFF7DDFD4FEA481141F022
:10B970000201002001F0E201FEF7FEF806EB4603AB
:10B9800098447E4B53F8283001AAC01A80EAE0732D
:10B99000A3EBE07342F827300137DFE7012D35DDF7
:10B9A000022D019E029D08D1AE4201DD304628E005
:10B9B000284631469DF8002026E0AE42039F0EDD6A
:10B9C000BE4207DD304629469DF80120FFF752FDB3
:10B9D00030460DE0384631469DF800200EE0BD426D
:10B9E0009DF8002008DD28463146FFF743FD284634
:10B9F00039469DF8022007E038463146FFF73AFD08
:10BA000038469DF801202946FFF734FD0025A3782C
:10BA10002B41DF0720D55A4B584AD3F8033003EBAC
:10BA200043032B44002652F82320514BEE54514B34
:10BA3000EE54514B01211878A94020EA0101EFB2E0
:10BA400019707901304601F0E001FDF7E0FD304664
:10BA500039463246FDF7A0FE0135032DD7D101F05E
:10BA600011BB802F7FF48DAE0025A3782B41DE071C
:10BA700024D5434B414AD3F8033003EB43032B4413
:10BA8000284652F82380FFF74DFD394B0026EE542F
:10BA9000384BEE54384B01221978EFB2AA4021EA14
:10BAA000020279011A70304601F0E0014246FDF7CA
:10BAB000AEFD304639463246FDF76EFE0135032DA8
:10BAC000D3D101F0DFBA02283FF65BAE142E3FF768
:10BAD00058AE400140F0020101F0E2010020FEF703
:10BAE0004BF8D4F80320A378244902EB42021A440D
:10BAF000002551F8226006441846FFF713FDA1788F
:10BB00001B4B5D541B4B5D541B4B012218788A4024
:10BB100020EA020249011A702846324601F0E0018B
:10BB2000FDF775FD2846A1782A46FDF735FE01F0A0
:10BB3000A9BA03232B7001F0A5BAFEF7FDFC01F0B2
:10BB4000A1BAFEF7F9FF01F09DBA7B789A1F012A8E
:10BB50000AD98C2B08D0C02B06D0C72B04D003F1F8
:10BB60003402D2B2322A0DD8A2787AB109E600BFE7
:10BB700057CDFF1FC0CDFF1F31CDFF1FF8CEFF1FD8
:10BB8000ECCEFF1FBA78022A3FF6FBAD952B2BD8DF
:10BB9000932B80F095800D2B0BD80C2B80F0908090
:10BBA000052B78D001D8042B0AE0062B79D0072B7F
:10BBB00030E0862B6FD00BD8822B00F08780832B50
:10BBC00040F0F380A0780621FDF7FEFE01F05ABA9E
:10BBD0008C2B00F081808D2B40F0E780A0781A211B
:10BBE000FDF7F2FE01F04EBAC32B00F0A58022D87B
:10BBF000B52B7CD009D8993B012B00F2D680A078D8
:10BC00001821FDF7E1FE01F03DBAC12B7ED000F214
:10BC10008880C02B40F0C980A278D54B51015818BC
:10BC20000A300B44C01A023200EB4210997AFDF739
:10BC300083FA01F027BAD22B00F08A8013D8C72BE1
:10BC40002FD0CC2B40F0B180A378C94A58011118ED
:10BC50000E311044081A023300EB43100222FDF7A4
:10BC6000CAFA01F00FBAD62B00F08180FE2B00F04B
:10BC70008D80D42B40F09980A378BD4A58011118CB
:10BC800014311044081A023300EB43100422FDF76C
:10BC9000B2FA01F0F7B9A0780C21FDF795FE01F09A
:10BCA000F1B9A278B24B5101581809300B44C01AAF
:10BCB000023200EB4210597AFDF73EFA01F0E2B988
:10BCC000A0781421FDF780FE01F0DCB9A0780421F2
:10BCD000FDF77AFE01F0D6B9A378002B7FF451ADC1
:10BCE0004B20A4490122FDF786FA01F0CBB9A278D6
:10BCF0009F49500100F11803181A023200EB42105C
:10BD000019440422FDF777FA01F0BCB9A078984BEA
:10BD100003EB401340014830197AFDF70DFA01F0AA
:10BD2000B1B9A3789249981C400101EB4311042258
:10BD3000FDF761FA01F0A6B9A0788D4901EB401139
:10BD40004001443004310422FDF755FA01F09AB95C
:10BD5000A2788749500100F11003181A023200EB53
:10BD6000421019440422FDF746FA01F08BB9A3787A
:10BD70007F4A580111181C311044081A023300EB95
:10BD800043100222FDF737FA01F07CB9A378784A14
:10BD9000580111180C311044081A023300EB4310FB
:10BDA0000122FDF728FA01F06DB903232B7001F091
:10BDB00069B97B789A1F012A0AD98C2B08D0C02B2D
:10BDC00006D0C72B04D003F13402D2B2322A02D8F3
:10BDD000A27822B1D5E4BA78022A3FF6D2AC952BEC
:10BDE0003ED8932B80F0BE800D2B0DD80C2B80F00D
:10BDF000B980052B00F08D8001D8042B0CE0062BB8
:10BE000000F0A180072B43E0862B00F082801BD836
:10BE1000822B00F0B780832B40F02F81A078062181
:10BE2000FDF7AEFDA578690141F0060101F0E601DC
:10BE30000020FDF799FC504B504A43F82500A378A9
:10BE40000021D15401F01EB98C2B00F0A1808D2B64
:10BE500040F01381A0781A21FDF792FD01F012B98C
:10BE6000C32B00F0D18024D8B52B00F0A88009D8CE
:10BE7000993B012B00F20181A0781821FDF780FD8C
:10BE800001F000B9C12B00F0A98000F2B280C02BF4
:10BE900040F0F380A378364A5C0111190A3114444A
:10BEA000081B023300EB4310FDF71FFAA07201F0EC
:10BEB000E9B8D22B00F0B48013D8C72B43D0CC2BD9
:10BEC00040F0DB80A3782A4A580111180E31104443
:10BED000081A023300EB43100222FDF71FFA01F0AB
:10BEE000D1B8D62B00F0AB80FE2B00F0B780D42B5E
:10BEF00040F0C380A3781E4A580111181431104431
:10BF0000081A023300EB43100422FDF707FA01F090
:10BF1000B9B8A0780C21FDF733FDA578690141F08F
:10BF20000C0101F0EC010020FDF71EFC144B134A3C
:10BF300043F82500A0780021115453F82010FDF794
:10BF40008FFC01F09FB8A378094A5C0111190931EF
:10BF50001444081B023300EB4310FDF7C6F960726E
:10BF600001F090B8A0781421FDF70AFD01F08AB81D
:10BF7000C8CDFF1FD3CDFF1F20D4FF1FBCC6FF1F9E
:10BF800014D0FF1FA0780421FDF7FAFC01F07AB865
:10BF9000A378002B7FF4F5AB8D4C4B2004F10B0103
:10BFA0000122FDF7BBF98B4B987804EB4014E17A42
:10BFB000C1F10801C9B2FEF767F801F063B8A278D1
:10BFC0008549500100F11803181A023200EB4210A3
:10BFD00019440422FDF7A2F901F054B8A0787E4C70
:10BFE00004EB401440014830FDF77FF9207201F066
:10BFF00049B8A3787849981C400101EB4311042209
:10C00000FDF78CF901F03EB8A078734901EB4011BF
:10C010004001443004310422FDF780F901F032B8C8
:10C02000A2786D49500100F11003181A023200EB9A
:10C03000421019440422FDF771F901F023B8A378E6
:10C04000654A580111181C311044081A023300EBDC
:10C0500043100222FDF762F901F014B8A3785E4A9A
:10C06000580111180C311044081A023300EB431028
:10C070000122FDF753F901F005B803232B7001F0FD
:10C0800001B8BB78022B00F09E80032B00F0B28039
:10C09000002B40F00A817B78502B6AD026D8472BA2
:10C0A0005BD012D8422B50D007D8402B48D0412B20
:10C0B00040F0F980494B1B78F3E0452B48D04AD833
:10C0C000442B40F0F080454BD8E04C2B4AD007D8A9
:10C0D000492B44D04B2B40F0E680404BDB78E0E02E
:10C0E0004E2B3E4B41D042D85B7DDAE0802B4ED0C8
:10C0F00013D8532B43D006D8512B3DD0522B40F0B0
:10C10000D280364BBDE0552B3ED03AD3562B40F073
:10C11000CA80324B93F82430C3E0832B40D006D83A
:10C12000812B37D0822B40F0BE802D4BA6E0852B93
:10C130003AD037D3FF2B40F0B6802A4B1B783EE035
:10C1400040F2FF70FDF7D1F886E0244B5B78A8E061
:10C15000224B5B79A5E0214B73E0204B6EE01F4B37
:10C16000DB7D2CE01D4B9B789BE0DB8C99E05B7EBC
:10C1700097E01A4B9B7D94E0184B1B7D91E0174B89
:10C1800062E0164B9B7E8CE0144BDB7E89E0144B07
:10C190001B7E86E0124B1B7E181F4342434180E00A
:10C1A0000F4B48E0104B43E00D4A104993684B4356
:10C1B00003F540533933936023F0004371E00033BB
:10C1C00018BF01236DE07A78094B53F8223068E0FC
:10C1D000C8CDFF1FECCEFF1FC8CDFF1F0CC0FF1F37
:10C1E000BCC6FF1F02D0FF1F04D0FF1F6D4EC6410B
:10C1F00020D0FF1F7B782E2B55D8DFE803F0181BCB
:10C200001E545454545454212427545454545454B4
:10C210005454545454545454542A2F3133353754AD
:10C2200054545454543B3E4144474A4D50009E4B55
:10C230001B6836E09C4B5B6833E09B4B9B6830E0AF
:10C24000994BDB682DE0984B1B692AE0964B5B69A4
:10C2500027E00020FDF745FC686028E0002006E0AC
:10C260000120F7E7012002E00220F3E70220FDF7BA
:10C270004DFCF1E78C4B9B6913E08B4BDB6910E0C5
:10C28000894B1B6A0DE0884B5B6A0AE0864B9B6A10
:10C2900007E0854BDB6A04E0834B1B6B01E0824BBC
:10C2A0005B6B6B6003E0032300E004232B707F4B88
:10C2B0001B78002B00F0E6867D4B6A681A607D4B88
:10C2C0002AB91A6842F008021A6000F0DBBE1A6848
:10C2D00022F008021A6000F0D5BEBB78022B16D1FE
:10C2E000754B5B78372B0ED8744903F5A770800027
:10C2F00001EB83010422FCF77EFF00F0C3BE7B78D4
:10C30000142B40F2D88203232B7000F0BBBE042311
:10C310002B7000F0B7BEBB78022B0DD17B78372B8A
:10C32000F1D8664903F5A770800001EB8301042270
:10C33000FCF7F4FF00F0A6BE04232B7000F0A2BEB1
:10C34000B87802283FF61DAA5B4B5B78012B07D01B
:10C3500002D3022B08D01EE002F0F3F800F092BEE8
:10C3600002F0F8F800F08EBE02F0FCF84F4B686067
:10C370001B78002B00F086864D4B18604D4B1A68D9
:10C3800020B942F008021A6000F07CBE22F00802D8
:10C390001A6000F077BE03232B7000F073BEBB78E9
:10C3A00013B1022B05D01CE03046FCF7A3FC00F0D3
:10C3B00069BE7878072808D81EB9FCF781FB00F021
:10C3C00061BEFCF759FB00F05DBEFF2840F05A86C5
:10C3D000711C0ABF364BF0B21878FCF795FB00F0E1
:10C3E00051BE042388F8003000F04CBEBB78012B0E
:10C3F00017D02BB1022B18D17878FCF7CBFB0EE0CD
:10C400007878082802D8FCF790FB08E00A2802D1C7
:10C4100000236B600BE0FF2809D1FCF7F1FB68609B
:10C4200005E0787802F0F0F8F9E704232B701F4B51
:10C430001B78002B00F026861D4B6A681A601D4B86
:10C440002AB91A6842F008021A6000F01BBE1A6886
:10C4500022F008021A6000F015BE7A78144B092AFF
:10C4600033D8DFE802F005080B0E12181B1E2D3121
:10C470001A68164428E01A68961B25E01A68564385
:10C4800022E01A6892FBF6F61EE01A6892FBF6F1BB
:10C4900006FB112618E01A68164015E01A681643C4
:10C4A00012E01A6856400FE038CEFF1F03D0FF1F7E
:10C4B000F4CFFF1FF4CEFF1FECCEFF1F20D0FF1FD5
:10C4C0001A68D2431A6000E01E601A689A4B2AB9B3
:10C4D0001A6842F008021A6000F0D4BD1A6822F00F
:10C4E00008021A6000F0CEBD944B1A68924BB2421B
:10C4F000196804DD21F0030141F0040108E00BBFDD
:10C5000021F0060121F0050141F0010141F0020195
:10C5100019602AB91A6842F008021A6000F0B2BD28
:10C520001A6822F008021A6000F0ACBD7B780C2B70
:10C5300000F2A885DFE803F0071019222B343E47EC
:10C540005059626B74007C4B1B681A0740F19A8546
:10C550007B4BDE6100F096BD774B1B681B0700F13B
:10C560009185774BDE6100F08DBD734B1B68DF0753
:10C5700040F18885724BDE6100F084BD6E4B1B6814
:10C58000DD0700F17F856E4BDE6100F07BBD6A4BFD
:10C590001B685C0740F17685694BDE6100F072BD77
:10C5A000654B1B6813F0050F00F06C85644BDE6172
:10C5B00000F068BD604B1B68980740F16385604BD5
:10C5C000DE6100F05FBD5C4B1B68990700F05A8587
:10C5D0005B4BDE6100F056BD574B1B68DA0640F13D
:10C5E0005185574BDE6100F04DBD534B1B689B06D8
:10C5F00040F14885524BDE6100F044BD4E4B1B6854
:10C600005F0640F13F854E4BDE6100F03BBD4A4B7B
:10C610001B681D0640F13685494BDE6100F032BDD6
:10C62000454B1B68DC0540F12D85454BDE6100F074
:10C6300029BD434BDE6100F025BD414B1A6A072A34
:10C6400000F22085511C03EB82021962D969516204
:10C65000DE6100F017BD3A4B1A6A002A00F012851D
:10C66000013A1A6203EB8202526ADA6100F00ABDF3
:10C670007B782E2B04D8334A0121D15400F002BD1F
:10C68000FF2B7FF440AE2E4B012283F8442000F0B4
:10C69000F9BC7B782E2B04D82A4A0021D15400F013
:10C6A000F1BCFF2B7FF42FAE254B002283F84420F2
:10C6B00000F0E8BC224D95F8453083B9701C4FF06E
:10C6C0000A0304D11D4A16687343AB6401E05E435C
:10C6D000AE64FCF719F80123E86485F84530637807
:10C6E000042B00F2CF84DFE803F0034C7BB0190089
:10C6F000FCF70AF8EA6CA96C114B801A80EAE07228
:10C70000A2EBE0728A4204D9002283F8452000F0AF
:10C71000B9BCDA69013ADA6100F0B4BCA07801F082
:10C7200021FF88B9044B85F845001A6822F01002F1
:10C730001A6000F0A7BC00BFF4CEFF1FF4CFFF1FAC
:10C74000BCC6FF1F8ACEFF1FAB6CA64CA3B1FBF784
:10C75000DBFFE36CA26CC01A80EAE073A3EBE0732A
:10C76000934209D9002384F845309F4B1A6842F060
:10C7700010021A6000F086BCEB69013BEB6100F02F
:10C7800081BC0020FCF7D3FFA3785B00184110F0B8
:10C79000010609D0002385F84530934B1A6822F032
:10C7A00010021A6000F06EBCAB6C8E4C9BB1FBF7B4
:10C7B000ABFFE36CA26CC01A80EAE073A3EBE073FA
:10C7C000934208D9884B84F845601A6842F01002F9
:10C7D0001A6000F057BCEB69013BEB6100F052BC02
:10C7E00001AA00207C21FCF7A8FFA27802235200B6
:10C7F00003FA02F29DF8063012EA030709D000237B
:10C8000085F84530784B1A6822F010021A6000F063
:10C8100039BCA96C734C99B1FBF776FFE16CA66C3F
:10C82000401A80EAE071A1EBE071B14208D96E4B89
:10C8300084F845701A6842F010021A6000F022BCB9
:10C84000EB69013BEB6100F01DBC01AA00207C21DB
:10C85000FCF773FFA3789DF806205B0042FA03F310
:10C8600013F0010609D0002385F845305E4B1A68A5
:10C8700022F010021A6000F005BCAA6C594C92B16B
:10C88000FBF742FFE26CA16C801A80EAE072A2EB37
:10C89000E0728A4207D9544B84F845601A6842F026
:10C8A00010021A60EEE3EB69013BEB61EAE34D4BEA
:10C8B00000221A76E6E34D4A9778022F1AD84C4A9E
:10C8C0004C4C927E03EB4301394444F82160002A2A
:10C8D00000F0D883002B00F0D583013B0C20584397
:10C8E000042200F5C36002FB070004EB8101FCF7A2
:10C8F00082FCC7E3FF2F7EF444AF3E4E83B90C2584
:10C90000002405F20C6071192044214404220434EF
:10C91000FCF771FC0C2CF4D10C35FC2DF0D1B1E3FB
:10C92000002563780C205A1E504303EB4303E9189B
:10C9300000F5C36000EB850006EB810104220135A0
:10C94000FCF759FC032DECD19CE37B78142B3FF6CC
:10C95000DAACBA78022A19D803EB43031A44264BFF
:10C9600024491B7851F822206A60002B00F08A834A
:10C97000224B1A601C4B22B91A6842F008021A6056
:10C9800080E31A6822F008021A607BE3FF2A7EF433
:10C99000F8AE184E83B90C25002405F20C6071190D
:10C9A0002044214404220434FCF7B8FC0C2CF4D1BC
:10C9B0000C35FC2DF0D165E3002563780C205A1E60
:10C9C000504303EB4303E91800F5C36000EB850017
:10C9D00006EB810104220135FCF7A0FC032DECD10C
:10C9E00050E300BFBCC6FF1FF4CEFF1FECCEFF1FFD
:10C9F0000CC0FF1FF8CEFF1F03D0FF1FF4CFFF1F97
:10CA000094F801809F4FB8F1140F3FF67CACBE78CC
:10CA100031062DD50025A3782B41DA070FD5994B88
:10CA200069015E7841F00201002001F0E201FDF7AA
:10CA3000A3F806EB46062E44934B43F82600934B8F
:10CA40009B7E8BB163787BB15A1E0C20504303EB65
:10CA500043038D4A00F5C360E91802EB810100EB46
:10CA600085000422FCF7C7FB0135032DD3D109E370
:10CA7000022E3EF686AE710141F00201002001F067
:10CA8000E201FDF779F8814B7F4C9B7E08EB48086B
:10CA9000464444F82600002B00F0F4827B78002BFB
:10CAA00000F0F082BD78591E0C20484303EB43038D
:10CAB0000422E91800F5C36002FB050004EB8101C4
:10CAC000FCF799FBDEE27A78714B0A2A42D8DFE85C
:10CAD00002F0060B11161C24292E33383C006D4938
:10CAE0001A6809680A4403E06A491A680968521A10
:10CAF0001A602FE067491A6809684A43F8E76549F0
:10CB00001A68096892FBF1F2F2E7624A1968126842
:10CB100091FBF2F002FB1012EAE75E4A11681A6814
:10CB20000A40E5E75B4A11681A680A43E0E7594A98
:10CB300011681A684A40DBE7564A1168C943116018
:10CB400008E054491A680A6004E0524A18681168FB
:10CB5000196010601A68504B22B91A6842F0080236
:10CB60001A608FE21A6822F008021A608AE2484BC3
:10CB70001B68C7F80330FDF7DFFC83E27B78052BE9
:10CB800000F28082DFE803F003090F151B21424BFE
:10CB90001A6802F00F021A6074E23F4B1A6822F022
:10CBA00010021A606EE23C4B1A6822F020021A60F2
:10CBB00068E2394B1A6822F040021A6062E2364B92
:10CBC0001A6822F080021A605CE2334B1A6822F481
:10CBD00080721A6056E27B782E2B3FF694AB2F4A78
:10CBE00002EB83031E654DE22C4B2949D3F80C213F
:10CBF0000A602849D3F810210A60D3F81421264985
:10CC0000DA61D3F818210A60D3F81C2183F8452093
:10CC1000D3F82021DA64D3F824219A64204993F8C8
:10CC20002821885C08B101208854002283F82C2137
:10CC300028E2BA78022A3EF6A4AD124B5B78142B98
:10CC40003FF661AB03EB43031A44114B0E491B68DB
:10CC500041F8223016E200F0C1FE13E200F0C0FEFF
:10CC600010E200F0BEFE0DE200F0BCFE0AE200F0B1
:10CC7000BAFE07E200F0B8FE04E2084B00221A7682
:10CC800000E200BFECCEFF1FF8CEFF1F0CC0FF1F5D
:10CC9000F4CFFF1F10D0FF1FF4CEFF1FBCC6FF1F35
:10CCA0008ACEFF1F7B7813B1012B04D00CE0B14B6F
:10CCB00001221A76E6E140F2FE7296423EF661AD3E
:10CCC000AC4A1376D661DDE103232B70DAE1A94B80
:10CCD000002183F8441083F82C11A64A02F1500376
:10CCE0004FF0FF3043F82100A348002343540131A3
:10CCF0002F29F2D11376D361136282F845309F4A0F
:10CD000013609F4A13609F4A1360BBE11B7D9B0722
:10CD10000AD440F2FE739E423EF633AD954B042298
:10CD20001A76C3F83061ADE108232B70AAE1914B6C
:10CD300000221A76A6E1944C9B78944A237040F224
:10CD4000FE7301259E42157027D8914B1B7D13EA77
:10CD5000050722D1304601A9FCF712F99DF80430ED
:10CD600063709DF80530A3709DF80630E3709DF860
:10CD70000A3023719DF8093063719DF80830A37162
:10CD80009DF80730E37127722B46E15C227A01336C
:10CD90000A44082B2272F8D174E101230021E154E6
:10CDA0000133082B784AF9D1137813726AE17B7842
:10CDB000012B1DD00AD3022B2BD1744B01221A70E8
:10CDC000734B714A9B781370002319E06F4B01225B
:10CDD0001A706F4B6C4A9B7813706E4B1868002367
:10CDE0000133C118082B11F8011CD154F8D149E1C5
:10CDF0000422EA716B7156220623AA712B7141E15C
:10CE0000654901331944082B11F8091CD154F7D195
:10CE100038E103232B7035E17B78032B00F232815C
:10CE2000DFE803F0020E191D524B1A7EEA7193F8E7
:10CE30004520D3F83031AA711A0A6A712B7121E1A9
:10CE40004C4B1A7EEA7193F84520DB69AA711A0AE5
:10CE50006A712B7116E1494B1B686B6012E1484BFC
:10CE60001B686B600EE17B78002B40F00B81B9787A
:10CE7000002940F0078140F2D2439E4240F00281F7
:10CE800040F2FF70FCF758F9FCF7BBF80120FBF704
:10CE90001DFDF7E07A78414B02B101221A70404B38
:10CEA000E2781A70334B93F834113E4B19703E49B7
:10CEB00000230B703D490B703D4B19780A431A70E3
:10CEC000E0E07C7814B1012C11D01DE0042240F286
:10CED000FB7001A9FCF722FA019BD7F803209A42C4
:10CEE00006BF0123C8F80430C8F80440CAE0BB7884
:10CEF0002A2B06D140F2FB702E490422FCF77BF965
:10CF0000C0E003232B70BDE0032388F80030B9E0B4
:10CF10007B78032B63D8DFE803F00802545F154ADF
:10CF20000023D2F83811144610E0124BD3F8382100
:10CF3000092A07D8511CC3F8381103EB8203C3F840
:10CF40003C619FE009232B709CE001338B4200F091
:10CF50009980194A52F82300B0424FEA8305F4D170
:10CF60002A44481E834229D2506842F8040B0133F8
:10CF7000F7E700BFBCC6FF1F8ACEFF1FF4CFFF1F1D
:10CF800010D0FF1FF4CEFF1FF9CFFF1FF8CFFF1FF8
:10CF90000CC0FF1F08C0FF1F0080000030CDFF1F26
:10CFA0005BCDFF1F80CEFF1F5ACDFF1FB9CEFF1FE5
:10CFB00031CDFF1FEFCEFF1FF8C7FF1FC4F83801A8
:10CFC00060E0324A0023C2F83831314A00219950DA
:10CFD0000433282BF9D155E00A236B6052E0032378
:10CFE0002B704FE07B78812B7EF4CBABBA78294B4A
:10CFF000922A7EF4C6AB9A79A32A7EF4C2AB5A7900
:10D00000B42A7EF4BEAB1A79C52A7EF4BAABDB78BB
:10D01000D62B7EF4B6ABFBF716FFFBF775FB044689
:10D02000FBF772FB001B0028B8BF4042B0F57A7FC7
:10D03000F6DBFBF745FC184B00221A604FF0FF327D
:10D04000C3F87021C3F87022C3F87421C3F87422A6
:10D05000C3F87821C3F87822C3F87C21C3F87C2276
:10D060000E4B0F4A1A600120FBF730FC0AE040F239
:10D07000D2439E4206D1054B012283F8642101E090
:10D0800002232B7004B0BDE8F08100BFBCC6FF1FB7
:10D09000F8C7FF1FECCEFF1F10E000E000C0FF1F2D
:10D0A00078563412324AF8B500241460314A324BB3
:10D0B0001460324ADC61146083F845401F46650104
:10D0C000EDB245F006010020FCF756FD2C4B45F073
:10D0D0000C0143F824000020FCF74EFD294B43F8D7
:10D0E00024000134032CEAD1274BD97AC1F108017D
:10D0F0000020C9B2FCF7C8FF0023244A0021995040
:10D100000433B3F5806FF8D1214EB37E83B10C2583
:10D110000024204905F20C602944204421440422C3
:10D120000434FCF7FBF80C2CF3D10C35FC2DEFD1BB
:10D13000F37E3BB1002096F82410FCF771FB737D61
:10D1400093B10CE04FF4A764134920462144042214
:10D150000434FCF7E3F8B4F5C36FF5D1EAE7FBF765
:10D1600037FE08B1012300E000233B76F8BD00BF85
:10D17000F4CFFF1F10D0FF1FBCC6FF1FF4CEFF1F50
:10D1800020D4FF1F14D0FF1FC8CDFF1F20D0FF1FCA
:10D190000CC0FF1FF8CEFF1FE8CAFF1FF7B50F4CEA
:10D1A0000F4E86460F4694E80300C6F803300D4B39
:10D1B000B27000228DE803001A7086F800E07770E4
:10D1C000FEF7D0F9084A217882F865119DE803003E
:10D1D000636884E80300184603B0F0BD08D0FF1F61
:10D1E000ECCEFF1F03D0FF1FBCC6FF1FF7B51F4EBD
:10D1F00002460C4696E803008DE803001C4953786C
:10D200000B7093784B70D3788B7013798B71537943
:10D210004B7193790B71D379CB70164B00271F702C
:10D22000FEF7A0F9144B19786D46334671B9217099
:10D2300061703278A2707278E270F2792271B279FC
:10D2400062717279A2713279E27109E0012907D124
:10D250003A460A4911444978A1540132082AF8D1C2
:10D2600095E8030083E8030003B0F0BD08D0FF1F7A
:10D27000ECCEFF1F03D0FF1FF8CFFF1FF9CFFF1F1A
:10D28000014B93F865017047BCC6FF1F2DE9F043C1
:10D29000A84BA94C1B788FB063B1A84B1B78062B09
:10D2A00008D00A2B06D003F0EF030F2B1CBF00237E
:10D2B00084F8343194F83431A14E5A1E012A3BD8F7
:10D2C000A049012BCA68079214BF082307238DF8D1
:10D2D0001830327894F866318DF8193000238DF8C3
:10D2E0001A30C2B98B688DF82030974B8DF8272003
:10D2F00019788DF8211059788DF82210D9798DF888
:10D30000231099798DF8241059791B798DF82510FF
:10D310008DF8263009E0012A07D1013306AA8B498E
:10D320001A44595CD171082BF7D106A801F08EFA86
:10D33000002800F02A83A3E0032B1FD133788BB998
:10D34000804F814DB87897F801802A7880449044C6
:10D350006A789044EA799044AA7990446A79904432
:10D360002A7918E0012B40F08B800025774B585D1F
:10D370000135FBF703FA092DF8D181E0042B28D100
:10D38000704F714DB87897F80180002301226B70BF
:10D390002A706B6080449044FBF7F0F97878FBF7D3
:10D3A000EDF92878FBF7EAF96878FBF7E7F9E8790F
:10D3B000FBF7E4F9A879FBF7E1F96879FBF7DEF907
:10D3C0005FFA88F82879FBF7D9F94046FBF7D6F9D8
:10D3D00056E0072B32D133782BBB5A4B93F802E03F
:10D3E00093F801C0584B8DF800E01F785D78D8792C
:10D3F0008DF80270E644774499798DF803503D44E6
:10D400005A798DF8040028441B798DF805100144E1
:10D410008DF806200A448DF8073013448DF801C0BA
:10D420008DF8083029E0012B27D10023474A9A5C68
:10D430000DF803200133092BF8D11EE0082B1FD172
:10D44000414A002301205370107053603D4A8DF80B
:10D450000200917852788DF801200A4402448DF838
:10D4600000108DF803308DF804308DF805308DF8FC
:10D4700006308DF807308DF808206846FBF7E0FC91
:10D48000334B1A789846002A00F08B80314B324D8E
:10D490001B78013B062B00F28080DFE803F00404D8
:10D4A000257E7E7E5F00274A297893688DF830308C
:10D4B00080238DF831308A238DF8323000238DF8A7
:10D4C00033308DF834308DF835308DF836108DF8D6
:10D4D000293007218DF82A300AA8D3688DF8281042
:10D4E0000B9301F0B3F958E0164F2A78B87897F803
:10D4F0000190814409F10A099144FBF73FF97878DA
:10D50000FBF73CF98020FBF739F98A20FBF736F965
:10D510000020FBF733F90020FBF730F90020FBF780
:10D520002DF95FFA89F92878FBF728F94846FBF7C7
:10D5300025F932E002D0FF1FBCC6FF1FECCEFF1F53
:10D54000F8CFFF1F0CC0FF1F08D0FF1FF9CFFF1F30
:10D55000B9CEFF1F80CEFF1F5ACDFF1F914B2A78F7
:10D56000987859788DF80D10802301448DF80E308D
:10D570000A318A238DF80C008DF80F308DF81320B6
:10D5800000230A4403A88DF810308DF811308DF86F
:10D5900012308DF81420FBF753FC00232B7088F811
:10D5A0000030002384F83431337094F8643113B1BF
:10D5B0000120FBF78BF906A801F0D4F8054698B3D3
:10D5C000794B9DF820201A709DF821205A709DF803
:10D5D00022209A709DF823209A719DF824205A7178
:10D5E0009DF825201A719DF82620DA709DF81930D3
:10D5F00084F86631FBF788F86C4B6D4D18606D4B05
:10D6000000221A709DF81830227E072B0CBF0123D0
:10D61000022385F83431531E012B674B02D9052AAA
:10D6200040F09E800022BAE003A8FBF7BFF8064650
:10D6300000285BD0FBF7D2F808B184F8675194F862
:10D6400067119DF80C005A4A4B1CDBB22144092B90
:10D6500084F8673181F8680140F0B680002392F8C1
:10D66000681182F867314F4A5278914240F0AC809D
:10D670001A464F4D05F5B471595C01330A44082B25
:10D68000D2B2F6D195F8703193422BD1464B95F832
:10D6900069211A7095F86A215A7095F86B219A7071
:10D6A00095F86C219A7195F86D215A7195F86E2153
:10D6B0001A7195F86F21DA70FBF726F83F4B404A54
:10D6C0001860297E00231370032285F834214A1E36
:10D6D000012A85F86731384A02D9052918BF012384
:10D6E000137071E0042385F834316DE00AAD2846EB
:10D6F000FBF793FB00283AD033463246E95C01330E
:10D700000A44082BD2B2F9D19DF8301091422BD1A6
:10D71000254B9DF829201A709DF82A205A709DF8F3
:10D720002B209A709DF82C209A719DF82D205A710B
:10D730009DF82E201A719DF82F20DA70FAF7E4FF79
:10D740001E4B1F4A186000231370072284F83421EF
:10D75000227E511E01291946174B03D9052A01D0F3
:10D7600001221CE019702FE084F834312CE0237E74
:10D770000F4D013B012B27D8EB6940F2FE7293421B
:10D7800020D8FBF725FBE8B1E8690749431CEB61AA
:10D79000FBF7F6FB092385F83431074B01221A7099
:10D7A00012E000BF0CC0FF1FECCEFF1F70CEFF1FAA
:10D7B000BCC6FF1F20CDFF1F03D0FF1F78CEFF1F69
:10D7C0007FCEFF1F00232376237E714D042B04D1CF
:10D7D000704E3278170640F1AD8094F8343113F072
:10D7E000FB0F05D0082B03D0062B01D0FDF7BAFEA6
:10D7F00094F83431092B79D1FAF786FF644A664DE3
:10D80000D2682B68801A80EAE072A2EBE0729A423A
:10D8100008D9624B1A78012A04BF02221A70FAF75B
:10D8200073FFE060FAF770FF23696A68C01A80EA44
:10D83000E073A3EBE073934208D9584B5A78012A5E
:10D8400004BF02225A70FAF75FFF2061FAF75CFF0B
:10D850006369AA68C01A80EAE073A3EBE07393429D
:10D8600008D94E4B9A78012A04BF02229A70FAF71F
:10D870004BFF606194F84430002B37D0444B93F851
:10D880002C21002A32D145498B5C022B2BD1404BF5
:10D8900003F1500050F82200451C22D0404983F883
:10D8A00028210968C3F80C113E490968C3F8101112
:10D8B000D969C3F814113C49D8610968C3F8181133
:10D8C00093F84510C3F81C110022D96CC3F820113D
:10D8D00083F84520996CC3F82411012283F82C2188
:10D8E00004E000238B5401322F2ACCD194F8341158
:10D8F000274B092904D11A7E022A04BF05221A7671
:10D90000D4F83821224B002A3FD009293DD1197E75
:10D9100001293AD1D86900231D4901F59E7454F8B4
:10D920002340A04202D105230B762EE0013393421F
:10D93000F2D12AE095F8343113F0FB0F25D0082BF3
:10D9400023D0062B21D0194CD6F80330D5F830015E
:10D95000636040F2FE739842627012D83146FBF762
:10D9600021FCD5F830013146FBF78EFB30B1D5F8FC
:10D9700030310133C5F83031652300E007232370CF
:10D9800003E00723237000232B760FB0BDE8F0835C
:10D99000BCC6FF1FECCEFF1F38CEFF1F8ACEFF1F75
:10D9A000F4CFFF1F10D0FF1FF4CEFF1F08D0FF1FC2
:10D9B000704710B5074CFAF7A7FE2368C01AB0F5F8
:10D9C000FA7F05D9044B2022DA60FAF79DFE206029
:10D9D00010BD00BF2CD4FF1F00F00F4070477047F0
:10D9E0007047704770477047704770472DE9FF4791
:10D9F0009F4C237833B96FF000436360A360E3600A
:10DA000001232370257C9B4F4DB9E8B2FBF78DF8BD
:10DA100078550135082DF8D1954B01221A74272528
:10DA20000026F0B2FBF781F8BB5D83421AD0914B20
:10DA3000B21DF054904B53F82230022B05D0032B2B
:10DA40000AD0012B0ED168B106E058B98B4A515D5E
:10DA5000012907D1535505E0884B5A5D012A04BFBF
:10DA600002225A550136082E05F10105D9D1844EFE
:10DA7000F369C3B1834D2F78AFB9FAF745FE824BF6
:10DA80001B68C01AF3690028B8BF404298420AD9FF
:10DA90003846FBF7BDFF0120FBF7BAFF0220FBF77A
:10DAA000B7FF01232B70336AD3B1784D2E78BEB9FE
:10DAB000FAF72AFE764B724A1B68126AC01A80EA8D
:10DAC000E073A3EBE07393420AD93046FBF7A0FF63
:10DAD0000120FBF79DFF0220FBF79AFF01232B702B
:10DAE0006C4D2B7B002B40F00782FAF70DFEE369AB
:10DAF000C01A80EAE073A3EBE0730A2B04DC664BE8
:10DB00001B69D80700F17C8294F82000584F002848
:10DB100040F00C810A21FBF727FE064697F820000B
:10DB2000DFF87881FCF7B4F836BB97F8201049018C
:10DB300041F00801304601F0E801FBF715FED8B9C5
:10DB4000FAF7E2FD97F8203007EB83024FF00A0E58
:10DB50005268801A05EB43120028B8BF4042918BEF
:10DB60000EFB01F1884227DD1846917AFAF7BCFED8
:10DB700097F8203001211DE094F8200058F830304B
:10DB800086EAE672A2EBE6729A4204D2434B03EBBA
:10DB9000C003197902E005EB4013597AFAF7A4FEA5
:10DBA00094F82070FAF7B0FD04EB870794F8203062
:10DBB000786000213A4AD15494F82000DFF8B0A0F0
:10DBC00058F83030354F86EAE679A9EBE679994581
:10DBD0000BD2FCF757FB9AF8203007EBC3077A7992
:10DBE00082420ED11846002109E0FCF74BFB9AF85F
:10DBF000203007EBC3077979884202D01846FCF73A
:10DC000015FB94F82000274B194F03440093264B33
:10DC100003440193254B002103EB80030A46FCF7E4
:10DC2000F3FB94F8200005EB40139B69C3B1FBF7AD
:10DC30009BF8A8B197F82000164B03EB40139B69A3
:10DC400099450DD9FBF7E4FE97F82030184A0121D9
:10DC5000D1540F33094AD15C012904BF0221D154A8
:10DC600056B394F82060134B9B5D8BBB58E000BF0C
:10DC700030C8FF1F41C8FF1F38CEFF1F8ACEFF1FCD
:10DC80000CC0FF1F7FCEFF1F78CEFF1F20CDFF1FD0
:10DC900070CEFF1FC8CDFF1FC0F00F403CCDFF1F4F
:10DCA00081CEFF1F38CDFF1FC3CDFF1F5CCDFF1FEF
:10DCB000C0CDFF1F84CEFF1F94F82010490141F012
:10DCC0000801304601F0E801FBF74EFD0028C8D1FD
:10DCD00094F8203005EB4312D28912B9B54AD35CCF
:10DCE00023B3FAF711FD94F8203004EB830205EB1F
:10DCF0004315526AE989801A80EAE072A2EBE07269
:10DD00000A2041438A4211DDAB4DEA5C72B91846E4
:10DD1000FCF7DCFBA94B93F820300122EA5405E024
:10DD2000FAF7F2FCA54B03EB860670620020FBF7C6
:10DD3000FEFC94F83020A14B8DF8080002F0F802A8
:10DD4000C10748BF42F0010283F83020430705D5E0
:10DD500094F8303043F0020384F83030C70605D51C
:10DD600094F8303043F0040384F83030944EDFF8F8
:10DD700070C2DFF870E2934F934B94F830809CF8B8
:10DD800000109EF800203878357893F80090B2465D
:10DD9000002341FA03F6F60713D548FA03F6F6070F
:10DDA0000FD542FA03F6F6070BD4012505FA03F660
:10DDB000F6B2B9F1000F46EA000046EA020208BFD7
:10DDC00000210133032BE4D194F830303870D807A8
:10DDD0008CF800108EF800208AF800500AD5774A97
:10DDE00092F83120D10705D4784AD178012904BFAF
:10DDF0000221D1709A0709D594F83120970705D4EC
:10DE0000724A1179012904BF022111715E0709D5F7
:10DE100094F83120550705D46C4A5179012904BF83
:10DE20000221517194F8202084F831300323B2FB91
:10DE3000F3F304A90B4413F9083C002B4ADA52010E
:10DE400042F01601002001F0F60103AAFBF775FC71
:10DE50009DF80E3058060BD5584A92F82010022033
:10DE60001B2210FB012259498D5C012D08BF8854EB
:10DE700019060AD594F82010544A0E3112F81100F0
:10DE8000012804BF022002F81100DA060AD594F82E
:10DE9000201002201B2210FB01224C498D5C012D19
:10DEA00008BF88549B060AD594F82020474B0E32B1
:10DEB00013F81210012904BF022103F8121094F87C
:10DEC0002010490141F01601002001F0F60103AADB
:10DED000FBF766FB94F82000384D00F095F894F8B5
:10DEE00020300133DBB2032B88BF002385F82030BC
:10DEF000FAF70AFCE06183E00020354E354B84F8E8
:10DF000020000146009301960246334B2B4FFCF74D
:10DF10007BFA94F820003356304E002B04EB0003BC
:10DF200093F832301CDB022B01D1335C83B105EB5B
:10DF30004015697AFAF7D8FC94F82000FCF7D2FA79
:10DF400094F82030E218022182F832100022F254B4
:10DF500094F82050FAF7D8FB04EB850460604FE09A
:10DF6000012B04D194F82030F35C9BB948E0FAF718
:10DF7000CBFB97F8203007EB830705EB43137A6858
:10DF80009B8B801A0A2180EAE072A2EBE0724B437D
:10DF90009A42E7DD94F8200005EB4013997AFAF7EE
:10DFA000A3FC94F8200005EB4015AB7AE3B9FCF72D
:10DFB0008DFA1DE084CEFF1F87CEFF1F30C8FF1FE4
:10DFC000B9CEFF1F5ACDFF1F30CDFF1F8ACEFF1FD6
:10DFD000C3CDFF1F38CDFF1F5CCDFF1F7CCEFF1FC1
:10DFE0005BCDFF1F31CDFF1F335C0BB1FCF77AFA1D
:10DFF00094F820301C44012284F832200022F2548C
:10E0000004B0BDE8F08700BF2DE9F04F470185B0AF
:10E01000FDB2044645F07C0103AA0020FBF78DFB0E
:10E020004FF0010A61009DF80E20009102238B4001
:10E030000AFA01FA03EA020902EA0A020192BA4A5A
:10E04000D1190020097A11F0800F01F07F0B904662
:10E0500007D0FAF76AFDD0F1010A38BF4FF0000A85
:10E0600006E0FAF762FD10F1000A18BF4FF0010A4E
:10E070000BF1FF32072A00F26182DFE812F008009C
:10E080000800080008001701170117011701A74E23
:10E09000325D0F2A00F25282DFE812F050021000C7
:10E0A0004F013C007E01490052005F007300A40054
:10E0B000D400D9005002F300FC003A0245F01401EC
:10E0C00003AA06EB840645F006050020FBF735FBA6
:10E0D0009DF80D30736029460020FBF745FB214673
:10E0E000306102220020FBF757FB0020294640F256
:10E0F000FF72FBF77AFA002021460322FBF76EFB42
:10E10000ABF1020BBBF1010F884F94BF0223042334
:10E110003B5513E2019B002B00F01082002045F0DC
:10E120000201FBF729FD824B43F8240029E1B9F1F4
:10E13000000F00F003822046FBF76AFC0623FCE197
:10E140004744214600200322FBF748FB002045F00E
:10E1500008017A68FBF749FA4CE1B9F1000F40F089
:10E16000ED8145F008054744484629464A46FBF7F5
:10E170003CFA7A68484629465242FBF736FA0823A9
:10E18000DBE1B9F1000F00F0D98145F00201002078
:10E19000FBF7F2FC81460020024645F00801FBF740
:10E1A00024FA634B53F82420C9EB020243F82420DD
:10E1B000002021460322FBF711FB08EB0703002098
:10E1C0005A6845F00601FBF710FA002007F0E0015D
:10E1D0004A46FBF71CFA002021460246FBF7DCFA10
:10E1E0000923AAE10020FBF7A2FA00990841C10720
:10E1F00040F1A481002045F0080902464946FBF79A
:10E20000F4F9002021460222FBF7C6FA002002465C
:10E2100045F00201FBF7FBF9002007F0E0010246A0
:10E22000ABF1030BFBF7F3F9BBF1010F00F27B81BC
:10E230004744002021460222FBF7AEFA7A6800200C
:10E2400049460CE1B9F1000F40F0198176E1B9F1CE
:10E25000000F40F0738145F002014846FBF78CFC4B
:10E2600045F0080180464A464846FBF7BEF90222BF
:10E27000484607F0E00198FBF2F2FBF7C8F9484680
:10E280001FE10020FBF753FA009B1841C20740F141
:10E29000558148E106EB8407002045F006013A6904
:10E2A000FBF7A3F9002021463A7943E11F4E325D86
:10E2B0000F2A00F24381DFE812F0410110003D0017
:10E2C0005B006C008B0041019F0041014101D700C0
:10E2D000E400B9000A0138012B0145F0140103AA3A
:10E2E0000020FBF72AFA06EB84039DF80D205A6004
:10E2F000002021460222FBF74FFA002045F00601DC
:10E3000040F2FF72FBF771F9002021460322FBF770
:10E3100065FABBF1060F65D0BBF1080F62D0034B65
:10E3200004221A550AE100BFC8CDFF1F68C8FF1FAD
:10E3300024CDFF1FBBF1060F09D106EB840300209B
:10E340005A6802F00402214642F0010205E0BBF1E6
:10E35000080F04D1002021460322FBF73FFA0020DA
:10E3600045F0080158F80720FBF73FF90323E4E0E4
:10E37000ABF10503012B06D8019B23B1BBF1060FBE
:10E3800032D10423D9E0BAF1000F00F0D7800C237A
:10E39000D3E0BBF1050F09D106EB840300205A68D6
:10E3A00002F00402214642F0020205E0BBF1070F31
:10E3B00004D1002021460322FBF710FA58F8072069
:10E3C000002045F008015242FBF70FF90523B4E0A5
:10E3D000ABF10502012A09D8B9F1000F06D0BBF153
:10E3E000050F01D10223A8E00F23A6E0BAF1000F28
:10E3F00000F0A4800723A0E0BAF1000F40F09E8057
:10E40000ABF1070BBBF1010F0AD906EB84035046B1
:10E410005A6802F00402214642F00102FBF7DEF9DD
:10E420004744002045F008017A6819E0BAF1000F6E
:10E4300040F08480ABF1070BBBF1010F0AD906EB6A
:10E44000840350465A6802F00402214642F0020258
:10E45000FBF7C4F9474400207A6845F008015242AE
:10E46000FBF7C3F80A2368E0BAF1000F66D000207A
:10E4700045F00201FBF780FB06EB8403D8610B2318
:10E480005BE0BAF1000F59D145F002015046FBF7AD
:10E4900073FB08EB070381465A6883F80DA05046CA
:10E4A00045F00601FBF7B3F806EB84030222DB69B3
:10E4B0009944504607F0E00199FBF2F2FBF7A7F808
:10E4C000504621460246FBF767F90D2335E0002050
:10E4D000FBF72DF900990841C3072FD500200E2323
:10E4E00045F0080102463355FBF77FF8214600202E
:10E4F0000222FBF751F9002045F002010246FBF72A
:10E5000086F8002007F0E0010246FBF780F815E0EE
:10E51000002021460222FBF73FF9002045F00801C8
:10E520000246FBF762F80E2307E006EB84030020A7
:10E530001A792146FBF752F90023335505B0BDE89F
:10E54000F08F034B1A5C0AB901221A54704700BFBE
:10E5500068C8FF1F024B1A5C0AB10F221A54704799
:10E5600068C8FF1F014B185C704700BF68C8FF1FD9
:10E57000124B1A68684620F0070102F01F028D4610
:10E58000052A01B509D0062A0DD0042A0FD1196930
:10E590000B4A89B2118045220AE01969084A89B2FA
:10E5A0009180462204E01969054A89B251804422CB
:10E5B000BDE801401A608546704700BF00B00B40BF
:10E5C00090C8FF1F0E4B41F230023A20995841F09B
:10E5D0000061995041F23C02995841F00061995014
:10E5E00003F5E8230C229A6006491022DA60002223
:10E5F0005A620A624A628A6244221A6000F090BA41
:10E600000070044000B0044009282BD8DFE800F077
:10E6100005080D1013162A2A1A20134B188801E03A
:10E62000114B5888C0F30B1070470F4B9888F9E7CF
:10E630000D4B188804E00C4B588801E00A4B988871
:10E6400080B27047084B58884FF4987380B203E04B
:10E65000054B9888342380B258434FF6FF7390FBE4
:10E66000F3F070470020704790C8FF1F30B541F2AB
:10E670003C032E4CE55845F01005E5502C4B4FF46B
:10E6800000749C646FF4F875DC64A3F51833A4F18E
:10E690003E542C441C604FF400545C60254C1C60BC
:10E6A0001C68E401FCD50138072813D8DFE800F026
:10E6B000100E0C0A081206041F480CE01F480AE05E
:10E6C0001F4808E01F4806E01F4804E01F4802E01A
:10E6D0001F4800E01F4858601F4B002058631F4828
:10E6E00018601F488D044FF080642840C3F88040B4
:10E6F000C3F884003AB11A48C3F89040940420400B
:10E70000C3F8940001E0C3F890204FF08464C3F88C
:10E71000A0401148C3F8A41022B1C0F8B040C0F81E
:10E72000B42030BDC0F8B02030BD00BF0070044040
:10E7300000A004400F0080508320FC018720FE02CF
:10E740008720FE0B8720FE0E8720FE1D8720FE4AB5
:10E750008720FE958720FE05004002400F008000C4
:10E760000000FC1F384BD3F88020C2F30362022A5A
:10E7700010B513D0D3F89020C2F30362022A0FD051
:10E78000D3F8A020C2F30362022A0AD0D3F8B03033
:10E79000C3F30363022B54D1032202E0002200E002
:10E7A0000122120102F1402303F50033D3F8801057
:10E7B000C1F303410170D3F8801011F4801118BF28
:10E7C00001218170D3F8801011F4001118BF0121CC
:10E7D0004170417821B9D3F88410C1F38A4103E034
:10E7E000D3F8841021F0604102F1402202F500329A
:10E7F0004160D2F88840240E0472D2F88840240C7C
:10E800004472D2F88840240A847202F18801D2F856
:10E810008820C2724A68120E02734A68120C427350
:10E820004A68120A82734A68C273D3F8802092023F
:10E830004CBF4FF084624FF08062C3F8802001200B
:10E8400010BD002010BD00BF00400240204BD3F897
:10E850007021C2F303620C2A38D04178426811B1AA
:10E86000C2F3110202E091041A4A0A40C3F874216B
:10E87000427A037A120442EA0362C37A1A43837A21
:10E8800042EA0322124BC3F87821427B017B120437
:10E8900042EA0162C17B0A43817B42EA0122C3F85A
:10E8A0007C2143788278002B14BF4FF042634FF0F5
:10E8B00040630AB143F480130278120402F4702218
:10E8C0001343034A0120C2F870317047002070479B
:10E8D000004002400000FC1F0B4B4FF00062C3F8E9
:10E8E00070214FF48022C3F87421084AC3F87821BC
:10E8F0006FF48471A2F166320A44C3F87C21044AA1
:10E90000C3F87021704700BF0040024078563412AF
:10E910000000080C684620F007018D460E4901B53D
:10E920004FF480430D48C1F8A03000220023C0E915
:10E9300000230B4A002313600A4A13600A4AD36477
:10E940005360D364094B1B7813B94FF480738B6306
:10E95000BDE80140854670470090044070CDFF1F20
:10E9600028CEFF1F34CDFF1F0090034030D4FF1F7F
:10E9700010B9024B09011960704700BF6CCDFF1F31
:10E98000B8B911F0040F0B4B08D04FF48042C3F814
:10E99000A020CA064CBF084A084A01E04FF4807222
:10E9A00001F008019A6301F0FF02054B01B1012259
:10E9B0001A7070470090044000010A00000109002D
:10E9C00030D4FF1F30B9044BD3E90023100A40EACA
:10E9D000036070470020704770CDFF1F70B50C4674
:10E9E0000646D0B9F9F76CFF0C492246E317C1E996
:10E9F0000023D1E900452B0243EA14632202C1E956
:10EA00000023074B1E60074B1E60074BDE645E60F1
:10EA1000DE64BDE87040F9F751BF70BD70CDFF1FD7
:10EA200034CDFF1F28CEFF1F0090034038B52B4A7E
:10EA30002B4D41F23C030024D15841F00071D150DC
:10EA4000284B5A6D42F004025A651A6822F01802E7
:10EA50001A605A6D22F001025A65D3F8842042F000
:10EA6000C002C3F884204FF6FF72DC645C609A60D9
:10EA7000D3F8802042F00102C3F88020D3F8802030
:10EA800042F02002C3F88020D3F8802042F0100228
:10EA9000C3F880205A6D42F001025A651A6842F0AC
:10EAA00008021A604FF4E0632B636B630E4B196925
:10EAB0000E4B4A091201204601F01F011A60FFF7B0
:10EAC0005FFF20462146FFF789FF4FF48043C5F8DA
:10EAD000A0305720BDE8384000F022B80070044054
:10EAE0000090044000900340C8CDFF1F6CCDFF1F75
:10EAF000FEE74FF0E023084AC3F8082D074A4CF21E
:10EB00002053D3814DF62813D381138823F00103BA
:10EB10001B041B0C13807047008000000020054080
:10EB2000802810B54FF00101154A06DD00F01F00E6
:10EB30008140C2F88C11D16010BD402806DD00F084
:10EB40001F008140C2F88811916010BD20280C463A
:10EB500006DD00F01F008140C2F88411516010BD35
:10EB6000084B0340002B03DA013B63F01F03013322
:10EB7000034A04FA03F3C2F88031136010BD00BFEA
:10EB800000E100E01F000080802810B54FF0010276
:10EB9000134905DD00F01F008240C1F88C2010BD34
:10EBA000402805DD00F01F008240C1F8882010BD1C
:10EBB0002028144605DD00F01F008240C1F88420A3
:10EBC00010BD084B0340002B03DA013B63F01F0329
:10EBD0000133034A04FA03F3C2F8803010BD00BFCA
:10EBE00000E100E01F000080064B1A78D2B2012A33
:10EBF00005D1222902D0212901D100225A700122F7
:10EC00005A707047A4C8FF1F70B5144611B91B4B4A
:10EC1000197070BD022903D1184B01221A7070BD02
:10EC2000042914D1154B5B78012B25D1958800233D
:10EC3000402D28BF40255E1CDBB2AB4205D22268C6
:10EC4000D05C00F0C7F83346F5E7002007E0032961
:10EC50000CD10A4B5A78012A0ED10020987002215B
:10EC600002460346BDE8704000F046BF052903D1C7
:10EC7000024B00221A705A7070BD00BFA4C8FF1F5B
:10EC800010B50446204600F0BDF80028FAD110BDAA
:10EC9000704710B5084C02460B4600200121A170B8
:10ECA00000F0EEFA224618B10023A370122010BD26
:10ECB0009378002BFCD110BDA4C8FF1FF8B5064601
:10ECC0000F4600F0FAFC0E4B1A78012A16D15B7839
:10ECD000012B13D100F000F988B10025ECB2BC4241
:10ECE00005D330462146BDE8F840FFF7D2BF3019C2
:10ECF00000F0D6F801350028F0D0F2E70C20F8BD7E
:10ED0000A4C8FF1F08B540210248FFF7D7FF00F055
:10ED100095F808BDA7C8FF1F38B5054600F0A8F84C
:10ED20000B28044609D106484021FFF7C7FF28B940
:10ED30002846BDE8384000F09BB80024204638BD86
:10ED4000E7C8FF1FF8B5002406460F462546A3B2C4
:10ED50009F4207D0305DFFF7DFFF002818BF0B256B
:10ED60000134F4E72846F8BD38B5451E002415F8EF
:10ED7000010F28B1FFF7D0FF002818BF0B24F6E7DA
:10ED8000204638BD07B50123002000930549064BF6
:10ED9000024600F01FFA002814BF1B20002003B019
:10EDA0005DF804FB09EC0000E9EB000038B50D4606
:10EDB000044600F097F885420AD825440020AC426A
:10EDC00007D020B914F8010B00F052F8F7E738BD6E
:10EDD0000B2038BD10B50A4B197840290ED05A784F
:10EDE0009C180132D2B2402AA07001F101014FF00B
:10EDF0000000197014BF5A70587010BD0B2010BD60
:10EE000027C9FF1F10B50C4B197891B193F8422018
:10EE10009C180132D2B2A4780470402A4FF000004E
:10EE200001F1FF31197014BF83F8422083F84200CA
:10EE300010BD0A2010BD00BF27C9FF1F014B187865
:10EE4000704700BF27C9FF1F024B1878C0F1400070
:10EE5000C0B2704727C9FF1F034B00225A7083F8C6
:10EE600042201A70704700BF27C9FF1FFFF7F4BF89
:10EE700010B50A4B197840290ED05A789C180132E7
:10EE8000D2B2402AA07001F101014FF000001970C8
:10EE900014BF5A70587010BD0B2010BD6AC9FF1FF7
:10EEA00010B50C4B197891B193F842209C1801329F
:10EEB000D2B2A4780470402A4FF0000001F1FF3173
:10EEC000197014BF83F8422083F8420010BD0A2055
:10EED00010BD00BF6AC9FF1F014B1878704700BF03
:10EEE0006AC9FF1F024B1878C0F14000C0B27047DA
:10EEF0006AC9FF1F034B00225A7083F842201A7020
:10EF0000704700BF6AC9FF1FFFF7F4BF70B5044622
:10EF1000007801F08DF901780023DAB28A4208D234
:10EF200003EB8305054466786D78AE4203F1010377
:10EF3000F3D1154D207A342303FB0253D97810B94D
:10EF400098780130987034235A43AB189B788B42E1
:10EF50000DD003F003030C2101FB03220A4B1A44DA
:10EF6000131D107951791B89926800F091FBD5F837
:10EF70009C3043B1227A002A224614BF0521032186
:10EF800012F8080B984770BDB0C9FF1F2DE9FF4765
:10EF90000D4691468DF80F0001F04AF9022D064604
:10EFA00049D190F800A00024E3B2534504F10104D4
:10EFB00009DA03EB830333440DF10F005978DA7853
:10EFC00001F0F6F9F0E74FF000085FFA88F75745CF
:10EFD00027DA07EB870737447C1C6078A3787978B9
:10EFE000B4F803200090002001900DF10F0001F013
:10EFF000BDF96378032B05D19DF80F007978184A85
:10F0000001F03CFA7978A37841F0100141EAC3118C
:10F010000DF10F00C9B2002201F0FAF908F1010860
:10F02000D3E7104BD3F89C30B3B19DF80F002946BD
:10F030004A46984710E0002DF3D12B463278591CF0
:10F04000DBB29A42EDD9074A342000FB03230022A9
:10F050009A70DA700B46F1E704B0BDE8F08700BFA4
:10F060000DEF0000B0C9FF1F2DE9F0410C7804F04E
:10F070006004202C1D4638D14C78042C1CD00AD8B2
:10F08000012C2ED02DD3022C1FD0032C29D1BDE86A
:10F09000F04100F05FB9212C1BD005D8202C20D1E5
:10F0A000BDE8F04100F03EB9222C16D0232C18D137
:10F0B000BDE8F04100F046B902241C801468002528
:10F0C00025701468671C17606570BDE8F04100F09A
:10F0D0005BB9BDE8F04100F01DB9BDE8F04100F0BA
:10F0E0007BB900202880BDE8F081402C06D1054C7A
:10F0F000D4F8A04014B1A047BDE8F081CD20BDE810
:10F10000F08100BFB0C9FF1F73B50446007801F05D
:10F110008FF863680093A27A637A43EA0223ADF81A
:10F12000043001780023DAB28A4208D203EB830567
:10F13000054466786D78AE4203F10103F3D1164DB4
:10F14000207A342303FB0253D97810B99878013020
:10F15000987034235A43AB189B788B420DD003F040
:10F1600003030C2101FB03220B4B1A44131D1079DE
:10F1700051791B89926800F08BFAD5F89C304BB11D
:10F18000227A20781AB1052104F1080201E0032156
:10F190006A46984702B070BDB0C9FF1F07B5436803
:10F1A0000093437A817A43EA0123ADF80430084B97
:10F1B000D3F89C30024643B1017A007811B10521A1
:10F1C000083201E004216A46984703B05DF804FB69
:10F1D000B0C9FF1F2DE9F8430546884617469946F2
:10F1E00001F026F802789DF8203001320646002111
:10F1F0002846D2B201F09CF8044630BB2846144998
:10F20000144A00F08EF93378601CE4B2A34211D99D
:10F2100004EB8402324434235C430F4992F801E04A
:10F2200001F804E00B1992785A7000229A70DA7093
:10F230000446E8E72846494600F066F8044620B947
:10F24000054BC3F89C80C3F8A0702046BDE8F88346
:10F250008DEF000069F00000B0C9FF1F08B5074B33
:10F260000022C3F89C20C3F8A02000F0ADF918B923
:10F27000BDE8084001F072B808BD00BFB0C9FF1F6B
:10F280002DE9F047914607460D46984600F0D0FF1D
:10F2900002780024E3B2934207D2013404EB8401E4
:10F2A000014411F8041CA942F4D1164A34205843F1
:10F2B0001118CE788B78F41AE4B2042C02D1C12054
:10F2C000BDE8F08706F003044FF00C0C0CFB0404BF
:10F2D00014440136F6B227716571C4F80890A4F899
:10F2E0000C80CE70F61AF6B2012E07D138462946A8
:10F2F0004A464346BDE8F04700F0CAB90020BDE8E1
:10F30000F08700BFB0C9FF1F014B00201960704794
:10F3100054CAFF1F024B0979197100F08DBF00BF5D
:10F3200054CAFF1F13B5002402AA1C80044B42F8E4
:10F33000041D0979197100F08DFF02B010BD00BFE6
:10F3400054CAFF1F00201880014B4A88DA8070479A
:10F3500054CAFF1F30B50C460221198021796488F8
:10F36000084D012C297103D1BDE8304000F08ABF5F
:10F37000022C03D1BDE8304000F090BF002018807F
:10F3800030BD00BF54CAFF1F30B50C4602211980A2
:10F3900021796488084D012C297103D1BDE83040E2
:10F3A00000F088BF022C03D1BDE8304000F094BFCC
:10F3B0000020188030BD00BF54CAFF1F044B054A0F
:10F3C00019791B7A1171137203210A23FFF758BFB1
:10F3D00054CAFF1F4CC0FF1F70B500261E808B78DB
:10F3E0000E4CC3F340014A00637261F3000203F064
:10F3F0000103A37205462272FFF7E0FF23685BB1A9
:10F40000617A01F0020101F0FF02284611B12221C8
:10F41000324600E021219847002070BD54CAFF1FEA
:10F4200008B50246034B12F8080B1B6805219847E4
:10F4300008BD00BF60CAFF1F38B5084D04462A1D2D
:10F44000012100F0CDFF20460121802200F0E0FFE5
:10F450002B6820780A210022984738BD60CAFF1F18
:10F4600037B501210DF10702044600F0B9FF9DF800
:10F470000730074D802B04D1204601212A7900F066
:10F48000C7FF2B6820780B210022984703B030BDBE
:10F4900060CAFF1F436805215A7800F0B9BF73B5F1
:10F4A0000122002405460126002100F081FF334699
:10F4B00021468DE850002846102200F057FF2146D3
:10F4C0002246284600F074FF234621468DE850006E
:10F4D0002846102200F04AFF31462846022200F05A
:10F4E00097FF32462846062100F092FF2246284622
:10F4F000902100F08DFF044B28781B68214622469E
:10F50000984702B070BD00BF60CAFF1F42783AB989
:10F51000C178C90141F0100101F0900100F078BFFD
:10F52000704773B50C468DF8070001F0FBF91F4ECC
:10F5300034600446002836D110211D4A9DF807008A
:10F5400000F09CFF122104461A4A9DF8070000F0C3
:10F5500095FF2043C4B21421174A9DF8070000F01C
:10F560008DFF2043C4B21321144A9DF8070000F018
:10F5700085FF2043C4B21721114A9DF8070000F00F
:10F580007DFF02AD2043C4B2162115F8010D0D4ACE
:10F5900000F074FF2043C4B201212846032200F08A
:10F5A00037FF03233371204602B070BD60CAFF1FCE
:10F5B0009FF4000095F4000039F4000061F40000AD
:10F5C0000DF5000021F4000037B502AC174B04F82C
:10F5D000010D0022102120461A6000F051FF122177
:10F5E0000546204600F04CFF2843C5B214212046B2
:10F5F00000F046FF2843C5B21321204600F040FF2B
:10F600002843C5B21721204600F03AFF2843C5B26F
:10F610001621204600F034FF284310F0FF0003D1EC
:10F620009DF8070001F08AF903B030BD60CAFF1FE2
:10F6300030B585B004AC012104F8090D0DF10E02BE
:10F64000204600F0CDFE204606210DF10F0200F00D
:10F65000C7FE9DF80E30802B16D19DF80F309B070A
:10F6600012D59DF8070000F0E1FD012805460BD1F9
:10F6700072B6204600F038FB0022204629468DF85D
:10F680000E2000F0C5FE62B69DF80E0005B030BD3C
:10F6900073B50E4615461C468DF80700FFF7C8FFE8
:10F6A000802807D00DF1070031462A46234600F096
:10F6B000B9FA00E0002002B070BD7047062812D8E9
:10F6C00080000129C0B204BF0230C0B2074AC0F3B3
:10F6D0004703122101FB03231A884FF6FF739A4256
:10F6E00008BFFF207047FF20704700BF68CAFF1F98
:10F6F0002DE9F041334D344C344E002785F800712C
:10F700004FF4107284F8400288462046FF2102F030
:10F7100069F9304639464FF48062C4F8446202F019
:10F7200061F995F80C3143F0800385F80C3195F8B8
:10F730000C21244B1206FAD4254AFF21117093F8AC
:10F740000C2142F0400283F80C21A3F52C331A68F7
:10F75000B8F1000F02D042F0004201E022F0004276
:10F760001A60184B320A02F0FE0283F89C20C6F39E
:10F77000074283F8B020360E164A83F8B460C4F806
:10F780004822102283F80821012283F89420BF2206
:10F7900083F8802093F8002102F07F0283F8002193
:10F7A00093F8842042F0010283F8842093F88420A7
:10F7B00042F0100283F8842084221A770020BDE8EA
:10F7C000F08100BF0020074068CAFF1F00D6FF1F5E
:10F7D00056C0FF1F00D8FF1F0D4B93F80C2102F0FD
:10F7E000BF0283F80C21BF2283F8802093F8842085
:10F7F00002F0FE0283F8842093F8942002F0FE02C7
:10F8000083F894201A7F02F07B021A770020704759
:10F81000002007402DE9F3410B460D788C784549CF
:10F8200003C902AE06E90300B3F80310B1F5007F87
:10F8300003D90021D97002211971062D19D8AF0002
:10F84000012CF9B201D10231C9B249083A484FF04E
:10F85000120C0CFB01FC00EB0C014FF6FF76B1F82B
:10F860000080B045064604D193F80180B8F1030F3B
:10F8700001D995205BE0012CFBD891F80F80B8F1FD
:10F88000FF0F04BF4FF0000881F80F80B3F803802A
:10F8900020F80C808A73CA7BD6F84802C1F80200AF
:10F8A00002F0010247EA44071743FFB2CF735A78C8
:10F8B0004A74D6F844220C7402EBC70CB3F80380E8
:10F8C000ACF80280CCF804004FF0080C02F837C006
:10F8D000CF7BB3F8038087F0010702EBC70CCCF8AD
:10F8E0000400ACF802804FF0480C02F837C0B3F8BF
:10F8F00003703844C6F8480234B9C97B12F83100A5
:10F9000060F07F0002F8310058780C4A02AB03EB3C
:10F9100084042DB254F8083C12F82510012818BFB1
:10F9200043F001030B43DBB202F82530002002B0A4
:10F93000BDE8F081F01B010068CAFF1FC02007402E
:10F94000084610B51146FFF7B9FEFF281CD00F4B33
:10F950001222C0F3470002FB0030D3F84432C27BCE
:10F9600013F8324004F07F0403F8324082F00101C2
:10F9700013F8312002F07F0203F831204FF0FF33FB
:10F980008372C372002010BDC42010BD68CAFF1F5F
:10F9900073B50D468DF80700084611461646FFF769
:10F9A0008DFEFF2804461FD0294632460DF1070080
:10F9B000FFF7C6FFC4F3470312210D4C59436318E8
:10F9C000D4F848221888121AC4F848222DB2094ADD
:10F9D000002002F825004FF0FF3262545A709A70EE
:10F9E000DA701A715A7100E0962002B070BD00BF43
:10F9F00068CAFF1FC02007402DE9F04180460E462F
:10FA0000084611461746FFF759FE0C4CC0F3470055
:10FA1000122303FB0040C57BFF2D0DD03A46404624
:10FA20003146FFF78DFF2DB2D4F8443213F835205C
:10FA300062F07B0203F83520BDE8F08168CAFF1F41
:10FA400010B5084600211446FFF738FE084B122275
:10FA5000C0F3470002FB0030D3F84432C27B03EB13
:10FA6000C2035A68136823605368636010BD00BF07
:10FA700068CAFF1F10B508460C461146FFF71EFE68
:10FA8000FF281AD024B2104B13F82430DBB213F045
:10FA90000C0F12D09B0712D40C4BD3F8443213F83E
:10FAA0003020D2090DD180F00100C0B213F83030FF
:10FAB000DB090CBF0020032010BD052010BD012074
:10FAC00010BD032010BD00BFC020074068CAFF1F43
:10FAD00008B5FFF7F3FD074B1222C0F3470002FB06
:10FAE0000030C27BFF2A04D0D3F84432002103F84F
:10FAF000321008BD68CAFF1F2DE9F04108460021F9
:10FB00001E461746FFF7DAFD244BC0F347001225C7
:10FB100005FB0035EC7BFF2C3CD0B5F80080D3F81A
:10FB200044121FFA88F24FF6FF739A4232D084F0E3
:10FB3000010311F83330C3F3C013D8B250BB4FEAFE
:10FB4000C40C8EB901EB0C033046A3F80280D5F843
:10FB500002205A6011F8343003F0400363F0770359
:10FB600001F83430BDE8F0812B736B7301EB0C03AB
:10FB70006E81964228BF1646C5F806705E805F60AB
:10FB800011F8343003F0400363F0770301F83430A8
:10FB9000BDE8F0819420BDE8F08100BF68CAFF1F76
:10FBA0002DE9F04107460C46084611461546FFF779
:10FBB00085FD1A4BC0F34700122606FB0036184697
:10FBC000F17BFF2927D022B2154B84B196F811C0E2
:10FBD000012D14BF18261426BCF1010F18BF46F0E2
:10FBE000010613F822C046EA0C0603F8226013F857
:10FBF00022606FF3410603F82260D0F844320022FD
:10FC000003F831203DB9384621462A462B46BDE847
:10FC1000F041FFF771BFBDE8F08100BF68CAFF1F68
:10FC2000C02007402DE9F84308460F4601219046C1
:10FC30009946FFF743FDFF2832D01B4AC0F3470027
:10FC4000122404FB0024D2F84452E67B15F8363027
:10FC5000DB0905EBC60223D139B2144B13F821108E
:10FC600001F0020101F0FF00D1B92188C4F806803B
:10FC70001FFA89F363818B42A8BF0B462073607320
:10FC80005380C2F804800FB9C82305E015F8363058
:10FC900003F0400363F0770305F83630BDE8F883DE
:10FCA0009320BDE8F88300BF68CAFF1FC02007404B
:10FCB000034B044883F8981001210A4600F0A8BBC2
:10FCC00000200740A8CCFF1F054B0648002283F800
:10FCD0009420802283F80C210121FF2200F098BBA0
:10FCE00000200740A8CCFF1F38B51A4B93F800211D
:10FCF00002F07F0283F8002193F80C2102F0DF026A
:10FD000083F80C2193F8802042F0200283F88020B1
:10FD100093F8842002F0DF0283F8842093F8942083
:10FD200002F0DF0283F8942093F8942042F004025A
:10FD300083F8942044F620641D46013CA4B200F0F0
:10FD40009DFE002CF9D195F8943003F0FB0385F863
:10FD5000943038BD002007402DE9FF47BA4CBB4D19
:10FD600094F84022039995F8803095F8847095F8BE
:10FD700090608DF80420002262F317210391012185
:10FD80008DF8062002928DF807208DF80C201F4078
:10FD90000DEB0102FF2304F510708DF801308DF892
:10FDA000053000F01DFB95F80C31D907F6B20FD5E0
:10FDB0009DF80130802B0BD195F8003103F07F03C3
:10FDC00085F8003195F80C3103F0DF0385F80C312C
:10FDD0007A0711D59D4B042093F8A41093F8A02026
:10FDE00083F8800004AB42EA012223F80E2D122092
:10FDF00001A9029300F056FBFB0749D5934D9248A9
:10FE00000123BF2785F8803085F8887095F89430F5
:10FE1000002643F0020385F89430FF2185F89860AE
:10FE20004FF4107285F8006101F0DCFD31464FF4AB
:10FE30008062D4F8440201F0D5FDD4F8443203F5D1
:10FE40000073C4F84832824BFF221A7095F8943040
:10FE500003F0FD0385F8943095F80C3143F040032E
:10FE600085F80C319F2385F88C7085F8843095F8DF
:10FE7000943003F0DF0385F89430102001A900F0DE
:10FE800011FB95F8943003F0DF0385F8943061E1BD
:10FE90003D0740F1F4806D4B082283F88020320941
:10FEA000C6F3C001062A8DF805208DF8071007D883
:10FEB000C6F3800303EB820319B10233DBB200E027
:10FEC000FF23D4F84452D90068185A084FF0120C96
:10FED0000CFB0244426802924088ADF80D00E07BC2
:10FEE00080F00100E07383F0010615F83330C3F3AE
:10FEF000801383F001039B0105F836309DF807302D
:10FF00009DF80590012B05EBC60843D1DFF840A111
:10FF1000B9F1000F14D19AF80090B9F1000F0FD188
:10FF2000FF2349464A4601A88AF80030FFF708FD3A
:10FF300005F8369001A849464A464B46FFF7DCFDD6
:10FF40009AF80030012B04D09DF80530002B00F00A
:10FF50008A80BDF80DC0A38960892288D4F8061074
:10FF600063449BB29842A38106D85FFA8CFC624539
:10FF70000CD1A47B012C09D11944C31A9342D8BFD8
:10FF80009AB2A8F80220C8F8041053E00291ADF824
:10FF90000D3068E0B9F1000F1DD16B5CC3F3830332
:10FFA0000D2B2B4B06D101218DF806101278D209AA
:10FFB0001A7010E01A78012A0DD1FF21197001A8DA
:10FFC0004946FFF7BDFC05F8369001A849464A4668
:10FFD0004B46FFF791FD62894FF6FF739A4242D07C
:10FFE000BDF80D00A1892388014489B29842A181FE
:10FFF00001D18A4209D86AB3B2FBF3F003FB1020A7
:020000021000EC
:1000000080B238BBA07B012824D1521A9A42D8BFB3
:1000100093B243B9D4F80220C8F8042088F802301B
:1000200088F8033006E0D4F80620A8F8023011441E
:10003000C8F8041015F8363003F0400363F0770376
:1000400005F8363014E000BF68CAFF1F00200740E3
:1000500056C0FF1FD4F8063002934FF0FF33ADF8BF
:100060000D10A372E3729DF8050001A900F01AFAC1
:100070003A4B93F8942002F0DF0283F89420B807FB
:1000800017D5364C022384F8803094F8883094F8E1
:100090008C201620134001A98DF80C3000F002FAD4
:1000A000BF2384F8883094F8943003F0DF0384F899
:1000B0009430F9061CD5294C202384F88030102375
:1000C00084F88030142001A900F0ECF994F80C3188
:1000D00043F0200384F80C3194F8003143F080039E
:1000E00084F8003194F8843043F0200384F884309D
:1000F000BA060DD5194C202384F88030132001A9AD
:1001000000F0D0F994F8843003F0DF0384F88430F1
:100110003B061FD5FF2301A810210DF102028DF827
:10012000053000F05DF99DF80230012B04D100226A
:100130008DF805208DF80730084C802384F8803036
:10014000172001A900F0AEF994F8943003F0DF0312
:1001500084F8943004B0BDE8F08700BF0020074069
:100160000B4611461A4601F03DBC00BF30B50329CD
:10017000039D049C1CD123B9164A2A6004222280C4
:1001800026E040F209418B4205D1022A4FF00003DC
:1001900003D9012201E001231A460F490C2000FB7C
:1001A0000313D9681B6951F8221029609B5C0EE08B
:1001B000072901D9CD2030BD074B03EB8102126A1C
:1001C0002A60002AF6D003EB4101B1F840302380C9
:1001D000002030BD57C0FF1FF81B0100012904D8C3
:1001E000034B5B5C137000207047CD20704700BF4D
:1001F000B4CCFF1F01299DBF024B00205A54CD20D3
:10020000704700BFB4CCFF1F01298CBF0020012024
:100210007047054B1A788A4204D05878431A5842DE
:100220005841704701207047B4CCFF1F0020704731
:1002300000487047481C0100012906D8044BC1EB57
:10024000C1011944116000207047CD20704700BFE4
:100250005BC0FF1F012910B50DD8094BC1EBC101CF
:10026000194408231068C45CC81801330F2B00F828
:10027000084CF7D101E0CD2010BD002010BD00BF1B
:100280005BC0FF1F012905D8034B03EB410111603F
:1002900000207047CD207047B6CCFF1F012905D83C
:1002A000034B03EB4101116000207047CD207047E4
:1002B000BACCFF1F01290AD80648136800EB410198
:1002C0001B788B7013685B78CB7000207047CD2053
:1002D000704700BFB4CCFF1F01290AD80648136835
:1002E00000EB41011B788B7113685B78CB710020A8
:1002F0007047CD20704700BFB4CCFF1F084B5A7821
:100300001A700023074AFF2199540133072BF9D1B2
:100310000023054A052199540133072BF9D1704771
:10032000BECCFF1FC0CCFF1FC7CCFF1F00BF704754
:10033000013AD2B2062A38B505461C4609D8064B02
:100340005A70FFF7DBFF28462146BDE83840FFF72B
:10035000CFB9992038BD00BFBECCFF1F024B002291
:100360005A70FFF739BA00BFBECCFF1F37B50F4C2C
:10037000257805B9B9B98DF802308DF800109DF8CF
:100380001830ADF8032000789DF81C208DF801305E
:100390006946FFF73FFA9DF800302BB120B923786A
:1003A000013B237000E0952003B030BDBECCFF1FA1
:1003B00038B50A4B0C461D7859788D421D4600D140
:1003C0004CB900782146FFF7E3FA2CB120B92B781D
:1003D00001332B7038BD962038BD00BFBECCFF1F47
:1003E0004B1E062B03D8094B19444B7808E0CB066B
:1003F00009D501F00F01062905D8044B19444B7AA1
:100400001370002070478220704700BFBECCFF1FD2
:100410004B1E062B2DE9F0418046154603D8164B9E
:1004200019444A7021E0CB0622D501F00F04062CB6
:100430001ED8012A4FEAD1160F4F04D12146324669
:10044000FFF7DAFA0FE072B93B195B7A012B0AD198
:1004500021463246FFF7A4FB2CB94046214686F0E0
:100460000102FFF79DFB3C4465720020BDE8F0816E
:100470008220BDE8F08100BFBECCFF1F0020704786
:10048000062903D9A1F11003072B07D8044B53F811
:100490002130002B14BF0020C4207047C4207047B7
:1004A000701C0100102838B504460D4601D1FFF735
:1004B00025FF044B53F824300BB128469847002001
:1004C00038BD00BF701C01001FB504A9144601F817
:1004D000090D02221A8008460DF10F020521FFF7CF
:1004E0007FFF034B9DF80F201A80236004B010BDDE
:1004F000D0CCFF1F1FB504A9144601F8090D012235
:100500001A8008460DF10F020421FFF769FF044B22
:100510009DF80F201A800020236004B010BD00BF9A
:10052000D0CCFF1F7FB500241C8049888DF80700C0
:10053000ADF80E10FFF768FE00B3BDF80E20114EA7
:10054000131B5A425A410DF107000121FFF760FFCA
:100550009DF80E200DF107000421FFF759FF736885
:100560000DF10E02054601219DF8070098477368BA
:100570009DF8070002212246984700E004252846FE
:1005800004B070BDD0CCFF1F37B502AA002402F81A
:10059000010D0D461C80104601210422FFF738FF93
:1005A0006A88024B20461A7203B030BDD0CCFF1FC0
:1005B00037B54C888D888DE80C00210AE2B22B46B5
:1005C000FFF7D4FD03B030BD2DE9F04186B00F46F2
:1005D0001E4600238DF80F000593904603230DF16E
:1005E0000F00012104AA8DF81030FFF7F9FE3D78C5
:1005F000274C15F0030525D106210DF111020DF14F
:100600000F00FFF7EDFE9DF811309DF80F0003F08D
:100610000303238005AB00930DF112030193022124
:100620002B462A46FFF7A2FD059BDB7913F0400F0E
:10063000238814BF43F0010323F001032380022326
:1006400033801FE0012D09D19DF81020BB88012ABD
:1006500002D113F0FF0F14D10023EFE7022D11D1C7
:10066000397941F010010DF10F00C9B20DF11202FC
:10067000FFF7B6FE9DF8123003F0010323803580AA
:1006800000E0CD20C8F8004006B0BDE8F08100BF12
:10069000D0CCFF1F7FB500221A800B784E788DF8E2
:1006A000070013F003030D46C6F3400632D1B6B17E
:1006B0004B88013B9BB2012B50D80DF1070006215E
:1006C0000DF10F02FFF78CFE0446002847D1AA78EF
:1006D0009DF80F3006FA02F21A43D2B211E04E88AA
:1006E000012E3BD10DF1070006210DF10F02FFF79E
:1006F00077FE044698BBAA789DF80F30964023EA0F
:1007000006020DF1070006218DF80F20FFF780FE8D
:10071000044624E0022B21D109798DF80F100DF148
:10072000070041F010013246FFF772FE6B78002E91
:100730000CBF08210721012B044607D19DF80F109B
:1007400001F00F00C909FFF7C3F90821054B9DF817
:1007500007005B680DF10F02984700E0CD242046AA
:1007600004B070BDD0CCFF1F10B500241C800B78E6
:1007700003F00303012B0A4605D109799278FFF7AC
:1007800039FD204610BD042010BD38B50C7804F0AA
:100790000304012C154607D11C80044C097922461C
:1007A000FFF71CFD2C6038BD042038BDD0CCFF1FE6
:1007B00013B5CD298DF8070006D10DF10700902162
:1007C0000122FFF725FE18E00D481C88018A1268F7
:1007D0008C4288BF198004461B889DF807000021C1
:1007E000FEF756FF94F90A30002B06DA00210DF1CE
:1007F00007000A460B46FFF77FF902B010BD00BFA5
:10080000D0CCFF1F73B5054600266A4601218DF83E
:1008100000600196FFF7E4FDAA783F4C012A46D11B
:1008200068680368C4F80A304368A07AC4F80E30D8
:1008300004F10A0110F0600F238A13D1E37A3748DC
:1008400050F82340002C5ED09DF80020022A5AD890
:1008500003EB43031844024492F83430012B52D185
:10086000287818E0202BADF802301AD873B10206B0
:100870000CD40A68C4F812204A68C4F81620284626
:10088000314604F11A02FFF737F943E0E46B002C1C
:1008900039D02878224901AA0DF10203A047014668
:1008A00032E002A82B7800F8073D902113E09DF874
:1008B0000030042B12D12B78217A02AD05F8063DC9
:1008C0002846FFF7F5F901210A462846FFF7A0FD63
:1008D000227A28460321FFF79BFD1BE094F90A309A
:1008E000002B17DBEB78ABB9E66B66B1B5F80930D6
:1008F00028780833ADF8023004F1120101AA0DF195
:100900000203B047CBE7CD21287801AA0DF10203FD
:10091000FFF74EFF02B070BDD0CCFF1FD01C01000E
:10092000DACCFF1F034B5960DA630021024AFFF75C
:10093000A5BD00BFD0CCFF1F0508010007B502AB65
:10094000054A03F8010D002118465160D163FFF7F5
:1009500097FD03B05DF804FBD0CCFF1F002070476B
:10096000354B41F24802995821F00D0141F0050143
:10097000995041F20402995841F48021995041F272
:100980003402995841F48021995003F52C336021A9
:1009900093F8942042F0020283F89420C02283F856
:1009A0000021FF221A7483F8802083F8882083F8BE
:1009B0008420002283F88C2083F80C111F491A75BB
:1009C000080A00F0FE0083F8982083F8C02083F81E
:1009D000C42083F8C82083F8CC2083F8D02083F883
:1009E000D42083F8D82083F8DC2083F8E02083F833
:1009F000E42083F8E82083F8EC2083F8F02083F8E3
:100A0000F42083F8F82083F8FC2083F89C00C1F3DD
:100A10000740090E83F8B00083F8B41083F8AC20C7
:100A20001A7783F8082193F8942002F0D40242F058
:100A3000010283F8942070470070044000D6FF1F25
:100A4000024B4FF400729A60704700BF00E100E073
:100A5000034B4FF40072C3F888219A60704700BFBF
:100A600000E100E010B5FEF78DF9044618B9FFF774
:100A7000EFFF204610BD1B2010BD00BF034B4AF204
:100A800002629A814BF280429A81704700200540B1
:100A900081F0004102E000BF83F0004330B54FEA2F
:100AA00041044FEA430594EA050F08BF90EA020F9C
:100AB0001FBF54EA000C55EA020C7FEA645C7FEA2F
:100AC000655C00F0E2804FEA5454D4EB5555B8BF52
:100AD0006D420CDD2C4480EA020281EA030382EAC3
:100AE000000083EA010180EA020281EA0303362D55
:100AF00088BF30BD11F0004F4FEA01314FF4801C28
:100B00004CEA113102D0404261EB410113F0004F39
:100B10004FEA03334CEA133302D0524263EB4303F0
:100B200094EA050F00F0A780A4F10104D5F1200E8E
:100B30000DDB02FA0EFC22FA05F2801841F10001E9
:100B400003FA0EF2801843FA05F359410EE0A5F1BD
:100B500020050EF1200E012A03FA0EFC28BF4CF0EE
:100B6000020C43FA05F3C01851EBE37101F00045A4
:100B700007D54FF0000EDCF1000C7EEB00006EEBB1
:100B80000101B1F5801F1BD3B1F5001F0CD349083B
:100B90005FEA30004FEA3C0C04F101044FEA445292
:100BA00012F5800F80F09A80BCF1004F08BF5FEA19
:100BB000500C50F1000041EB045141EA050130BDF9
:100BC0005FEA4C0C404141EB010111F4801FA4F19C
:100BD0000104E9D191F0000F04BF01460020B1FAF1
:100BE00081F308BF2033A3F10B03B3F120020CDA29
:100BF0000C3208DD02F1140CC2F10C0201FA0CF007
:100C000021FA02F10CE002F11402D8BFC2F1200C6B
:100C100001FA02F120FA0CFCDCBF41EA0C01904021
:100C2000E41AA2BF01EB0451294330BD6FEA04046A
:100C30001F3C1CDA0C340EDC04F11404C4F1200255
:100C400020FA04F001FA02F340EA030021FA04F367
:100C500045EA030130BDC4F10C04C4F1200220FABE
:100C600002F001FA04F340EA0300294630BD21FAFC
:100C700004F0294630BD94F0000F83F4801306BFC2
:100C800081F480110134013D4EE77FEA645C18BFB6
:100C90007FEA655C29D094EA050F08BF90EA020F4D
:100CA00005D054EA000C04BF1946104630BD91EA45
:100CB000030F1EBF0021002030BD5FEA545C05D148
:100CC0004000494128BF41F0004130BD14F5800487
:100CD0003CBF01F5801130BD01F0004545F0FE41FB
:100CE00041F470014FF0000030BD7FEA645C1ABF30
:100CF000194610467FEA655C1CBF0B46024650EA67
:100D0000013406BF52EA033591EA030F41F4002192
:100D100030BD00BF90F0000F04BF0021704730B518
:100D20004FF4806404F132044FF000054FF00001ED
:100D300050E700BF90F0000F04BF0021704730B5AE
:100D40004FF4806404F1320410F0004548BF404283
:100D50004FF000013EE700BF42004FEAE2014FEAD8
:100D600031014FEA02701FBF12F07F4393F07F4FB3
:100D700081F06051704792F0000F14BF93F07F4FE5
:100D8000704730B54FF4607401F0004521F0004128
:100D900020E700BF50EA010208BF704730B54FF0AE
:100DA00000050AE050EA010208BF704730B511F0B3
:100DB000004502D5404261EB41014FF4806404F1EB
:100DC00032045FEA915C3FF4DCAE4FF003025FEA6D
:100DD000DC0C18BF03325FEADC0C18BF033202EBF5
:100DE000DC02C2F1200300FA03FC20FA02F001FA4F
:100DF00003FE40EA0E0021FA02F11444C1E600BFEE
:100E000070B54FF0FF0C4CF4E06C1CEA11541DBFA0
:100E10001CEA135594EA0C0F95EA0C0F00F0DEF86B
:100E20002C4481EA030621EA4C5123EA4C5350EA50
:100E3000013518BF52EA033541F4801143F48013A1
:100E400038D0A0FB02CE4FF00005E1FB02E506F032
:100E50000042E0FB03E54FF00006E1FB03569CF087
:100E6000000F18BF4EF0010EA4F1FF04B6F5007F8D
:100E700064F5407404D25FEA4E0E6D4146EB0606FF
:100E800042EAC62141EA55514FEAC52040EA5E5088
:100E90004FEACE2EB4F1FD0C88BFBCF5E06F1ED832
:100EA000BEF1004F08BF5FEA500E50F1000041EB69
:100EB000045170BD06F0004646EA010140EA020016
:100EC00081EA0301B4EB5C04C2BFD4EB0C0541EA38
:100ED000045170BD41F480114FF0000E013C00F34D
:100EE000AB8014F1360FDEBF002001F0004170BD71
:100EF000C4F10004203C35DA0C341BDC04F114048A
:100F0000C4F1200500FA05F320FA04F001FA05F215
:100F100040EA020001F0004221F0004110EBD370E2
:100F200021FA04F642EB06015EEA430E08BF20EA0E
:100F3000D37070BDC4F10C04C4F1200500FA04F3B1
:100F400020FA05F001FA04F240EA020001F0004143
:100F500010EBD37041F100015EEA430E08BF20EAB6
:100F6000D37070BDC4F1200500FA05F24EEA020EFE
:100F700020FA04F301FA05F243EA020321FA04F02D
:100F800001F0004121FA04F220EA020000EBD370E4
:100F90005EEA430E08BF20EAD37070BD94F0000FE4
:100FA0000FD101F00046400041EB010111F4801F18
:100FB00008BF013CF7D041EA060195F0000F18BFC9
:100FC000704703F00046520043EB030313F4801F05
:100FD00008BF013DF7D043EA0603704794EA0C0FBF
:100FE0000CEA135518BF95EA0C0F0CD050EA4106D5
:100FF00018BF52EA4306D1D181EA030101F0004152
:101000004FF0000070BD50EA410606BF1046194679
:1010100052EA430619D094EA0C0F02D150EA013685
:1010200013D195EA0C0F05D152EA03361CBF1046C6
:1010300019460AD181EA030101F0004141F0FE4165
:1010400041F470014FF0000070BD41F0FE4141F4E9
:10105000780170BD70B54FF0FF0C4CF4E06C1CEAE9
:1010600011541DBF1CEA135594EA0C0F95EA0C0F9E
:1010700000F0A7F8A4EB050481EA030E52EA033559
:101080004FEA013100F088804FEA03334FF080557A
:1010900045EA131343EA12634FEA022245EA1115A7
:1010A00045EA10654FEA00260EF000419D4208BF58
:1010B000964244F1FD0404F5407402D25B084FEA05
:1010C0003202B61A65EB03055B084FEA32024FF4B1
:1010D00080104FF4002CB6EB020E75EB030E22BF0E
:1010E000B61A754640EA0C005B084FEA3202B6EBCE
:1010F000020E75EB030E22BFB61A754640EA5C007D
:101100005B084FEA3202B6EB020E75EB030E22BF0C
:10111000B61A754640EA9C005B084FEA3202B6EB0D
:10112000020E75EB030E22BFB61A754640EADC00CC
:1011300055EA060E18D04FEA051545EA16754FEA2E
:1011400006164FEAC30343EA52734FEAC2025FEA4C
:101150001C1CC0D111F4801F0BD141EA00014FF0DB
:1011600000004FF0004CB6E711F4801F04BF0143AC
:101170000020B4F1FD0C88BFBCF5E06F3FF6AFAEC8
:10118000B5EB030C04BFB6EB020C5FEA500C50F158
:10119000000041EB045170BD0EF0004E4EEA1131DB
:1011A00014EB5C04C2BFD4EB0C0541EA045170BDE2
:1011B00041F480114FF0000E013C90E645EA060E26
:1011C0008DE60CEA135594EA0C0F08BF95EA0C0F54
:1011D0003FF43BAF94EA0C0F0AD150EA01347FF49C
:1011E00034AF95EA0C0F7FF425AF104619462CE773
:1011F00095EA0C0F06D152EA03353FF4FDAE1046D6
:10120000194622E750EA410618BF52EA43067FF426
:10121000C5AE50EA41047FF40DAF52EA43057FF4B6
:10122000EBAE12E74FEA410212F5001215D211D5CA
:101230006FF47873B3EB625212D94FEAC12343F0D3
:10124000004343EA505311F0004F23FA02F018BF55
:10125000404270474FF00000704750EA013005D11E
:1012600011F0004008BF6FF0004070474FF00000E1
:10127000704700BF4FEA4102B2F1E04324BFB3F52B
:10128000001CDCF1FE5C0DD901F0004C4FEAC002FD
:101290004CEA5070B2F1004F40EB830008BF20F0E1
:1012A0000100704711F0804F21D113F13872BCBF9B
:1012B00001F00040704741F480114FEA5252C2F1F0
:1012C0001802C2F1200C10FA0CF320FA02F018BF39
:1012D00040F001004FEAC1234FEAD32303FA0CFC8C
:1012E00040EA0C0023FA02F34FEA4303CCE77FEA1B
:1012F000625307D150EA01331EBF4FF0FE4040F465
:101300004000704701F0004040F0FE4040F4000013
:10131000704700BF80F0004002E000BF81F0004154
:1013200042001FBF5FEA410392EA030F7FEA226C8B
:101330007FEA236C6AD04FEA1262D2EB1363C1BF1B
:10134000D218414048404140B8BF5B42192B88BF8A
:10135000704710F0004F40F4000020F07F4018BFAD
:10136000404211F0004F41F4000121F07F4118BFCD
:10137000494292EA030F3FD0A2F1010241FA03FC75
:1013800010EB0C00C3F1200301FA03F100F000435D
:1013900002D5494260EB4000B0F5000F13D3B0F125
:1013A000807F06D340084FEA310102F10102FE2A94
:1013B00051D2B1F1004F40EBC25008BF20F0010004
:1013C00040EA03007047490040EB000010F4000FB2
:1013D000A2F10102EDD1B0FA80FCACF1080CB2EB45
:1013E0000C0200FA0CF0AABF00EBC25052421843A4
:1013F000BCBFD0401843704792F0000F81F4000149
:1014000006BF80F400000132013BB5E74FEA41031B
:101410007FEA226C18BF7FEA236C21D092EA030F87
:1014200004D092F0000F08BF0846704790EA010F01
:101430001CBF0020704712F07F4F04D1400028BF2E
:1014400040F00040704712F100723CBF00F5000010
:10145000704700F0004343F0FE4040F40000704746
:101460007FEA226216BF08467FEA236301464202F2
:1014700006BF5FEA412390EA010F40F48000704705
:101480004FF0000304E000BF10F0004348BF4042AB
:101490005FEA000C08BF704743F0964301464FF0E7
:1014A00000001CE050EA010208BF70474FF0000343
:1014B0000AE000BF50EA010208BF704711F0004384
:1014C00002D5404261EB41015FEA010C02BF844654
:1014D0000146002043F0B64308BFA3F18053A3F5B3
:1014E0000003BCFA8CF2083AA3EBC25310DB01FAFA
:1014F00002FC634400FA02FCC2F12002BCF1004F7E
:1015000020FA02F243EB020008BF20F0010070470E
:1015100002F1200201FA02FCC2F1200250EA4C0062
:1015200021FA02F243EB020008BF20EADC707047A8
:101530004FF0FF0C1CEAD0521EBF1CEAD15392EAB6
:101540000C0F93EA0C0F6FD01A4480EA010C400292
:1015500018BF5FEA41211ED04FF0006343EA5010EC
:1015600043EA5111A0FB01310CF00040B1F5000F2E
:101570003EBF490041EAD3715B0040EA010062F1DD
:101580007F02FD2A1DD8B3F1004F40EBC25008BFC7
:1015900020F00100704790F0000F0CF0004C08BFE5
:1015A00049024CEA502040EA51207F3AC2BFD2F1B2
:1015B000FF0340EAC250704740F400004FF00003C0
:1015C000013A5DDC12F1190FDCBF00F000407047FA
:1015D000C2F10002410021FA02F1C2F1200200FA38
:1015E00002FC5FEA310040F1000053EA4C0308BFFF
:1015F00020EADC70704792F0000F00F0004C02BF50
:10160000400010F4000F013AF9D040EA0C0093F0CA
:10161000000F01F0004C02BF490011F4000F013B24
:10162000F9D041EA0C018FE70CEAD15392EA0C0F92
:1016300018BF93EA0C0F0AD030F0004C18BF31F0FD
:10164000004CD8D180EA010000F00040704790F0D3
:10165000000F17BF90F0004F084691F0000F91F077
:10166000004F14D092EA0C0F01D142020FD193EA3D
:101670000C0F03D14B0218BF084608D180EA0100C5
:1016800000F0004040F0FE4040F40000704740F0A1
:10169000FE4040F4400070474FF0FF0C1CEAD0526F
:1016A0001EBF1CEAD15392EA0C0F93EA0C0F69D0CB
:1016B000A2EB030280EA010C49024FEA402037D036
:1016C0004FF0805343EA111143EA10130CF000402D
:1016D0008B4238BF5B0042F17D024FF4000C8B421D
:1016E00024BF5B1A40EA0C00B3EB510F24BFA3EBFD
:1016F000510340EA5C00B3EB910F24BFA3EB9103CD
:1017000040EA9C00B3EBD10F24BFA3EBD10340EA26
:10171000DC001B0118BF5FEA1C1CE0D1FD2A3FF66C
:1017200050AF8B4240EBC25008BF20F00100704721
:101730000CF0004C4CEA50207F32C2BFD2F1FF03C4
:1017400040EAC250704740F400004FF00003013AF5
:1017500037E792F0000F00F0004C02BF400010F499
:10176000000F013AF9D040EA0C0093F0000F01F0AD
:10177000004C02BF490011F4000F013BF9D041EACF
:101780000C0195E70CEAD15392EA0C0F08D1420202
:101790007FF47DAF93EA0C0F7FF470AF084676E7D5
:1017A00093EA0C0F04D14B023FF44CAF08466EE7AE
:1017B00030F0004C18BF31F0004CCAD130F000427C
:1017C0007FF45CAF31F000437FF43CAF5FE700BFD4
:1017D0004FF0FF3C06E000BF4FF0010C02E000BFFD
:1017E0004FF0010C4DF804CD4FEA40024FEA41039F
:1017F0007FEA226C18BF7FEA236C11D001B052EA55
:10180000530C18BF90EA010F58BFB2EB030088BF1A
:10181000C81738BF6FEAE17018BF40F00100704789
:101820007FEA226C02D15FEA402C05D17FEA236C6B
:10183000E4D15FEA412CE1D05DF8040B704700BFB2
:10184000844608466146FFE70FB5FFF7C9FF002849
:1018500048BF10F1000F0FBD4DF808EDFFF7F4FF82
:101860000CBF012000205DF808FB00BF4DF808ED1B
:10187000FFF7EAFF34BF012000205DF808FB00BF3E
:101880004DF808EDFFF7E0FF94BF012000205DF860
:1018900008FB00BF4DF808EDFFF7D2FF94BF012011
:1018A00000205DF808FB00BF4DF808EDFFF7C8FF0A
:1018B00034BF012000205DF808FB00BF42000ED2BB
:1018C000B2F1FE4F0BD34FF09E03B3EB126209D47B
:1018D0004FEA002343F0004323FA02F070474FF031
:1018E0000000704712F1610F01D1420202D14FF0A6
:1018F000FF3070474FF00000704700BFFDF7F9F868
:10190000002100F004B80C4B5B58435004310B48E5
:101910000B4B42189A42FFF4F6AF0A4A00F003B8A4
:10192000002313600432084B9A42FFF4F9AF00F031
:101930000DF8804770470000641D010008C0FF1FBC
:1019400068C5FF1F00C6FF1F00DAFF1F224C08B545
:10195000F6F78BFDF6F7EEFDF6F7B0FFF6F7C9FFE9
:10196000F6F7BEFEF7F772FAFCF72CFEF7F7FBFC72
:10197000F7F75AF8E08CF7F753F92078F6F7CAFE34
:10198000E078F6F737FFF7F73DFA60792189228A88
:10199000FCF76CFEF8F740F9F8F72EFBFDF746F878
:1019A0000E4B04229A60FBF77DFBFCF701F80C4B11
:1019B00020229A60FBF76AFCFCF718F8FBF7F9FFA6
:1019C000F7F7DCF9F7F70EFA0028F3D0F8F714FB75
:1019D000FBF768FBEEE700BF0CC0FF1FC0F00F4035
:1019E00000F10F40F0B4840743D0541E002A3ED0CB
:1019F000CDB2034603E0621E002C38D0144603F833
:101A0000015B9A07F7D1032C2AD9CDB245EA052507
:101A10000F2C45EA054515D9A4F110073F0903F13C
:101A2000100606EB07161A46156055609560D560DE
:101A30001032B242F8D104F00F040137032C03EB4B
:101A400007130DD91E462246043A032A46F8045BC2
:101A5000FAD8221F22F003020432134404F00304D4
:101A60002CB1C9B21C4403F8011BA342FBD1F0BC4A
:101A7000704714460346C6E7024B13B1024800F014
:101A800005B8704700000000991A010001460020C7
:101A90000246034600F018B838B5094D094C641BDE
:101AA000A41018BF05EB840505D0013C55F8043D92
:101AB0009847002CF9D1BDE8384000F047B900BF85
:101AC000601D0100641D0100F0B5274C2668D6F8A2
:101AD000484185B00746002C41D065681F2D1EDDAA
:101AE000224818B94FF0FF3005B0F0BD4FF4C87070
:101AF000039102920193AFF300800399029A019B34
:101B000004460028EED0D6F84851256000206060D9
:101B10000546C6F84841C4F88801C4F88C013FB9AD
:101B2000AB1C00200135656044F8231005B0F0BD02
:101B300004EB85004FF0010CC0F88820D4F88861D0
:101B40000CFA05F21643022FC4F88861C0F8083178
:101B5000E6D1D4F88C311A43C4F88C21E0E706F5BD
:101B6000A674C6F84841B8E73C1D0100000000001B
:101B70008025000040380000004B0000807000000D
:101B80000096000000E10000002C010000C20100EE
:101B90000084030090D0030020A1070040420F0002
:101BA000F40100006400000001800808000000004B
:101BB000006400000000000000000000C8000000F9
:101BC0000000000000000000010003E80000000029
:101BD00000000003E800000000000200FA06000315
:101BE00000000000003706000000000000000000B8
:101BF000080000000400000057C0FF1F04000000A0
:101C0000090400005C1C01006C1C010000000000C5
:101C10000000000000000000000000002EC1FF1FB7
:101C2000EBC0FF1F000000000000000000000000EB
:101C3000000000000000000000001200430000004F
:101C40000000000000000000030102011000020279
:101C500000100003030110000001000057C0FF1F27
:101C6000B1C0FF1F8BC0FF1F69C0FF1F043A2622AF
:101C70000508010009F100009DF100000DEF0000D2
:101C80002D0301002D0301002D0301002D03010090
:101C90002D0301002D0301002D0301002D03010080
:101CA0002D0301002D0301002D0301002D03010070
:101CB0009FF4000039F4000095F4000061F4000086
:101CC00039F400002D03010021F400000DF500009F
:101CD000C9050100950601000000000095060100FD
:101CE0000000000089050100B105010000000000AE
:101CF000F5040100250501008B07010069070100BB
:101D0000C9040100010100010100000000010100FF
:101D100000000000010101010100000001010001BB
:101D200001000100000100000100000031313130EC
:101D300056313036000000004300000040C1FF1F54
:101D4000F8B500BFF8BC08BC9E467047F8B500BFA8
:081D5000F8BC08BC9E46704778
:081D5800791A01003584000036
:041D600011840000EA
:101D64002C1D010000010200000800000100000019
:101D7400020000000000000000000000000000005D
:101D84000000000000000000000007000000000048
:101D9400000000000000000000000000000000003F
:101DA40000000000A1200000000002000000FF0469
:101DB40003090400C2010000000800000000000044
:101DC400002203420041004400200053005400520A
:101DD4000049004E004700200049004E00440045E1
:101DE40000580026035300740065007000700065FD
:101DF40000720020004D006F0074006F007200201C
:101E04000044006500760020003A03540052004963
:101E1400004E0041004D004900430020004D006F7A
:101E240000740069006F006E00200043006F006EB4
:101E340000740072006F006C00200020002000205D
:101E440000200009024300020100C032090400001E
:101E5400010202000005240010010524010101040F
:101E640024020605240600010705830310000A095D
:101E7400040100020A0000000705810210000007A7
:101E840005020210000012010002020000103C2AA8
:101E94000001020001020001000000002CC4FF1F29
:101EA40094C4FF1FFCC4FF1F0000000000000000DA
:101EB400000000000000000000000000000000001E
:101EC400000000000000000000000000381D0100B8
:101ED40000000000000000000000000000000000FE
:101EE40000000000000000000000000000000000EE
:101EF40000000000000000000000000000000000DE
:101F040000000000000000000000000000000000CD
:101F140000000000000000000000000000000000BD
:101F240000000000000000000000000000000000AD
:101F3400000000000000000000000000000000009D
:101F440001000000000000000E33CDAB34126DE63A
:101F5400ECDE05000B0000000000000000000000A3
:101F6400000000000000000000000000000000006D
:101F7400000000000000000000000000000000005D
:101F8400000000000000000000000000000000004D
:101F9400000000000000000000000000000000003D
:1022C400641D010008C0FF1F60050000000000003D
:0822D400000000000000000002
:020000020000FC
:020000041FFFDC
:04C00000000000003C
:04000003100018FDD4
:00000001FF
